:020000040002F8
:10600000305C0020C1630200C9630200CB63020060
:10601000CD630200CF630200D163020000000000E4
:10602000000000000000000000000000D363020038
:10603000D563020000000000D7630200D9630200AC
:106040005D670200DB630200FD6A0200DB630200A1
:10605000DB630200DB63020095650200DB63020084
:10606000DB630200DB630200DB630200DB63020030
:10607000DB630200DB630200DB630200DB63020020
:10608000DB630200B5670200DB630200DB63020032
:10609000D9670200DB630200DD670200DB630200F8
:1060A000DB630200DB630200DB630200DB630200F0
:1060B000DB630200DB630200000000000000000060
:1060C000DB630200DB630200DB630200DB630200D0
:1060D000DB630200DB630200DB6302000000000000
:1060E00000000000000000000000000000000000B0
:1060F00000000000000000000000000000000000A0
:10610000000000000000000000000000000000008F
:10611000000000000000000000000000000000007F
:10612000000000000000000000000000000000006F
:10613000000000000000000000000000000000005F
:10614000000000000000000000000000000000004F
:10615000000000000000000000000000000000003F
:10616000000000000000000000000000000000002F
:10617000000000000000000000000000000000001F
:10618000000000000000000000000000000000000F
:1061900000000000000000000000000000000000FF
:1061A00000000000000000000000000000000000EF
:1061B00000000000000000000000000000000000DF
:1061C00000000000000000000000000000000000CF
:1061D00000000000000000000000000000000000BF
:1061E00000000000000000000000000000000000AF
:1061F000000000000000000000000000000000009F
:10620000DFF80CD000F088F900480047B5A802007C
:10621000305C002030B450E8012F93B2C48923448D
:106220008489A34228BF1B1B0489A34202BFBFF37A
:106230002F8F002007E0C3EA020340E80134002C5E
:10624000E9D14FF001000A6030BC704750E8012FDF
:10625000C2EA024240E801210029F7D1704730B478
:1062600050E8022F1FFAA2F3C488A34202BFBFF373
:106270002F8F00200DE0C48923448489A34228BFC6
:106280001B1BC2EA034340E80234002CE8D14FF064
:1062900001000A6030BC704750E8022FC2EA224277
:1062A00040E802210029F7D17047034653E8022F46
:1062B000D988B2EB324F4FF0000017BF92B241EADB
:1062C000014142EA014104E05A68B2EB324F08BF93
:1062D000012043E80212002AE8D1704730B4044696
:1062E00054E8000F0D4644E80053002BF8D1156028
:1062F00030BC704730B4044654E8000F40EA010552
:1063000044E80053002BF7D1156030BC704730B41F
:10631000044654E8000F00EA010544E80053002B4E
:10632000F7D1156030BC704730B4044654E8000F14
:1063300080EA010544E80053002BF7D1156030BC1A
:10634000704730B4044654E8000F00EB010544E800
:106350000053002BF7D1156030BC704730B40446B1
:1063600054E8000FA0EB010544E80053002BF7D1DF
:10637000156030BC704770B404464FF0000054E81C
:10638000006F0D68AE4207BF44E80023012044E8D7
:1063900000630E60002B1CBF0020F0E770BC70474C
:1063A00030B4044654E8000F88422CBF451A054615
:1063B00044E80053002BF5D1156030BC7047000055
:1063C0000648804706480047FEE7FEE7FEE7FEE78F
:1063D000FEE7FEE7FEE7FEE7FEE7FEE7E167020015
:1063E000016202002DE9F05F0546002092469B46BF
:1063F00088460646814640241BE0284641464746DB
:10640000224600F079F853465A46C01A914110D3FB
:1064100011461846224600F016F82D1A67EB0108BF
:106420004F4622460120002100F00DF817EB00092D
:106430004E41201EA4F10104DFDC484631462A46C5
:106440004346BDE8F09F202A04DB203A00FA02F11F
:10645000002070479140C2F1200320FA03F3194352
:1064600090407047004870476404030010B5431A19
:10647000934209D28318881803E010F8011D03F82D
:10648000011D521EF9D210BD40EA01039B0703D043
:1064900009E008C9121F08C0042AFAD203E011F863
:1064A000013B00F8013B521EF9D210BDD2B201E00F
:1064B00000F8012B491EFBD270470022F6E710B509
:1064C00013460A4604461946FFF7F0FF204610BD62
:1064D000421C10F8011B0029FBD1801A704730B50F
:1064E00004460020034600E05B1C934203D2E05CBC
:1064F000CD5C401BF8D030BD202A04DB203A21FAC5
:1065000002F00021704721FA02F3D040C2F12002CC
:106510009140084319467047064C074D06E0E06875
:1065200040F0010394E8070098471034AC42F6D3DA
:10653000FFF76AFE380C0300580C030070B58C1886
:1065400010F8015B15F0070301D110F8013B2A1187
:1065500006D110F8012B03E010F8016B01F8016B74
:106560005B1EF9D12B0705D40023521E0DD401F870
:10657000013BFAE710F8013BCB1A921C03E013F839
:10658000015B01F8015B521EF9D5A142D8D300206E
:1065900070BD00002DE9F04700268AB0DFF8509169
:1065A000B0464FF48075012437460696284605F01C
:1065B00061FA38B1D9F80403204203D0284605F027
:1065C0004FFA26432D1D64007F1CADB2082FEDD37A
:1065D0004FF4BE74204605F04DFA48B1204605F050
:1065E0003FFA46F0004606AA0121002005F024FAF1
:1065F000404D16F0FF0F15D00127002437420DD073
:1066000009EB8401D1F81005D1F81015C0F304206E
:1066100055F82420C1F3014102B190477F00641C6A
:10662000082CEBD3002E5FDA4FF0FF30CDF810804E
:1066300054E0281910F8507F90F9000027F0C008A6
:10664000401C3BD007A9404604F043FC10B34FEA7E
:106650009719404602F07AF955F820701FB1B9F148
:10666000030F03D006E0B9F1030F27D104A9404678
:1066700004F037FC4FF0A04101EB8800D0F8000790
:1066800006A9C0F3014A404604F023FC18B1BAF150
:10669000020F03D012E0BAF1030F0FD1B9F1030FCB
:1066A00008D1BAF1020F1DD00221404605F0A8F929
:1066B000761CF6B217B149464046B847641C042C14
:1066C000B7D3002E10D06A460121002005F0B4F99E
:1066D00006990098884207D0069004980026344610
:1066E0000790A6E70321E0E70AB0BDE8F0870000C5
:1066F000006000409833002000F01F02012191400B
:106700004009800000F1E020C0F88012704700F0DE
:106710001F02012191404009800000F1E020C0F8F3
:106720000011704700F01F020121914040098000D4
:1067300000F1E020C0F8001270474907090E002858
:1067400006DA00F00F0000F1E02080F8141D704719
:1067500000F1E02080F800147047000070B54FF49D
:106760008076304604F0F4FC114CB50560B130463B
:1067700004F0F5FC0120C5F80803607920B9012078
:1067800060712168002088474FF48276304604F01B
:10679000DFFC00280AD0304604F0E1FC0220C5F8F6
:1067A00008032168BDE870400120084770BD000063
:1067B000882C002007480021C0F84011C0F844117F
:1067C000C0F84811C0F84C11C0F80011C0F804110D
:1067D00008F06CBE0010014008F0B6BD05F0F0BE38
:1067E000F0B5B5480023021D0178101D01254FF0BA
:1067F000805406290BD11678360708D10678C6F3DF
:106800000316032E06D0042E04D0052E02D006292E
:1068100007D00EE0B4F82463A84FC6F304263E6008
:1068200002E01678360704D10678C6F30316032E65
:1068300002D0062904D00FE0A24FA14E7E670EE0E1
:106840001678360708D10678C6F30316032E06D04D
:10685000042E04D0052E02D0062907D00EE0D4F86D
:106860004462994FC6F342363E6002E0167836071E
:1068700004D10678C6F30316032E02D0062906D0EB
:1068800011E0924E376827F0807737600EE0167877
:10689000360708D10678C6F30316032E06D0042E59
:1068A00004D0052E02D006290AD011E04FF0804610
:1068B000C6F80C31C6F81031834E361F336002E043
:1068C0001678360704D10678C6F30316032E02D0D5
:1068D000062905D00CE07C4F032664373E600AE0B1
:1068E0001678360704D10678C6F30316032E02D0B5
:1068F00006290DD014E0764F05263E60744E78369A
:106900003560734E083633603F263F1D3E6002E01F
:106910001678360704D10678C6F30316052E02D082
:10692000062957D062E06B4E36686B4F3E60694E69
:10693000361D36683F1D3E60664E083636683F1D80
:106940003E60644E0C3636683F1D3E60614E103628
:1069500036683F1D3E605F4E143636683F1D3E6010
:106960005C4E183636685C4F20373E60594E1C36F8
:1069700036683F1D3E60574E203636683F1D3E60EC
:10698000544E243636683F1D3E60524E28363668D7
:106990003F1D3E604F4E2C3636683F1D3E604D4ECB
:1069A000303636684C4F40373E604A4E3436366893
:1069B0003F1D3E60474E383636683F1D3E60454EAF
:1069C0003C3636683F1D3E60424E403636683F1DBD
:1069D0003E6002E01678360708D10678C6F3031643
:1069E000032E06D0042E04D0052E02D0062907D08F
:1069F00019E0D4F85812394A01F04F01116002E051
:106A0000117809070FD10078C0F30310032803D0D1
:106A1000042801D0052806D131480168C90702D0F1
:106A20006FF001010160D4F83001062808D1D4F8D4
:106A30003401062804D12B48016841F480610160CB
:106A400022487438016841F470010160BFF34F8F30
:106A5000BFF36F8F4FF01021D1F80002002803DB45
:106A6000D1F80402002822DA1F4A15601F48046882
:106A7000002CFCD01524C1F800420568002DFCD084
:106A8000C1F8044201680029FCD0136001680029A4
:106A9000FCD0BFF34F8F0D48F0380168144A01F461
:106AA000E06111430160BFF34F8F00BFFDE7124962
:106AB00010480860F0BD0000E00F00F040350140D4
:106AC0000DF0ADBA00C007403C050040FCED00E011
:106AD000105600400404001020C50040E40E0040A1
:106AE000000400403C17004004E5014000E4014080
:106AF0000400FA050090D003AC2D00200148006886
:106B000000470000902C002002E008C8121F08C1B6
:106B1000002AFAD170477047002001E001C1121F1E
:106B2000002AFBD1704700000121202803DA8140B0
:106B30000548014003E0402802DA2038814009B1CD
:106B40000120704700207047FC06FFBD082806D2D0
:106B500028B1012803D0042801D00120704700206B
:106B6000704710B560B159B102780B785208B2EB9A
:106B7000530F05D10622401C491CFFF7B0FC08B199
:106B8000002010BD012010BD800701D000207047FB
:106B900001207047C3688B4206D811440069491E22
:106BA000814201D8012070470020704710B50122B2
:106BB0000221002001F0DAFC08B1072810D10722D9
:106BC0000221012001F0D2FC08B1072808D10021E0
:106BD0000A22084601F0CAFC08B1072800D10020AB
:106BE00010BD000010B550B10A480321008801EB28
:106BF000004009A105F02EF907F05CF903E003213C
:106C0000094800F06FFD002803D0BDE8104000F0F7
:106C1000CBB810BDF82D0020457261736520626FFE
:106C20006E647321000000000C2F002070B58CB042
:106C300015460E4600236C46C3F10F01415CE1543A
:106C40005B1C102BF8D30D2104F11000FFF735FC6D
:106C50000020C0F10F02315C2244401C1174032853
:106C6000F7D3684646DF0020C0F10F01214491F8B8
:106C700020102954401C0328F6D30CB070BD02200C
:106C800001F07EBB0149097900F080BF142C00207F
:106C900070B50024064D06E06868012110F8340044
:106CA00005F078FD641C28788442F5D3002070BD7F
:106CB000982C0020F8B515460C460646052A01D248
:106CC0000720F8BD05F062FE18B905F027FE002880
:106CD000F7D1124900224E600C708D60C1E9042288
:106CE000C1E906220E4D0DE006EBC40029680091B3
:106CF00081788DF8011000780A4A694605F09CFDFC
:106D00000028DED1641EE4B2EED2BDE8F8400448AB
:106D10000021054A001D00F053B80000982C002007
:106D2000DC000300959A0200398E020072B605F06D
:106D300047F900BF04F07EFF0028FBD1104C012171
:106D4000208801EB00400FA105F084F8104800688E
:106D5000C00700D000BE2088022101EB00400DA139
:106D600005F078F8BFF34F8F0948E43801680D4A01
:106D700001F4E06111430160BFF34F8F00BFFDE7F5
:106D8000F82D0020466174616C206572726F72008C
:106D9000F0ED00E053797374656D2072657365746E
:106DA000000000000400FA050EB500210091CDE9B5
:106DB00001106A4644F20100FFF7B8FF0EBD000063
:106DC000074B9B7823B12AB120B10068037C1BB12B
:106DD00008207047072070474174426100207047C7
:106DE0006434002070B507F0B5FB104800240B2177
:106DF000047044700E4D817014206C602C706C70A7
:106E0000FFF77AFC07211420FFF797FC1420FFF707
:106E10007EFC0848046007211120FFF78EFC05481E
:106E2000001F0068A860002070BD000064340020CE
:106E3000B82C0020081501402DE9FC47DFF87890B8
:106E400099F8023073B368B3052902D20720BDE870
:106E5000FC87436933B3437C012B25D000270446CC
:106E60000025884616468DF80050684600F038F830
:106E700001A808F0E9FDC8B1012101700F49446083
:106E80000968C0E90218C0E904769DF8040089F891
:106E900001009DF8000000F047F81420FFF742FCC5
:106EA0002846D4E70820D2E70F46D8E704259DF806
:106EB000000000F039F8F3E76434002004150140C5
:106EC0000649897839B130B1416921B10021017495
:106ED000022108F0C7BA082070470000643400207F
:106EE00030B5EFF3108172B60D4A9468012324B1D6
:106EF0000370002900D162B630BD93604FF0E023EB
:106F0000D3F88051074C25401560C3F88041D3F871
:106F1000844154605A17C3F8842100220270E8E7C4
:106F200070350020FC06FFBD0B498A68002A11D08D
:106F300000280FD1EFF3108072B60B684FF0E022FB
:106F4000C2F800314B68C2F8043100228A60002880
:106F500000D162B6704700007035002010B5144CA7
:106F600000224FF480312068FFF766FF08B1FFF779
:106F70001BFF00224FF400416068FFF75DFF08B17E
:106F8000FFF712FF002242F26661A068FFF754FF8C
:106F900008B1FFF709FF00224FF42031E068FFF746
:106FA0004BFF002803D0BDE81040FFF7FDBE10BD29
:106FB00074FF02002DE9F041064608680C46411CAA
:106FC0004FF0A0474FF0010506D005FA00F1C7F8D1
:106FD0000815206804F000FD6068411C02D0002103
:106FE00004F0E8FC3168A069C1F82405607D227DC9
:106FF00031681043C1F86C05D4E900123068C0F85C
:107000001425C0F80C15207D012815D1A068411C5D
:1070100002D0002104F0CEFCE068411C05D0854080
:10702000C7F80855E06804F0D7FCD4E902123068CC
:10703000C0F80825C0F81015BDE8F0812DE9F04131
:10704000064608680C46411C4FF0A0474FF001056A
:1070500006D005FA00F1C7F80815206804F0C6FC50
:107060006068411C02D0002104F0ADFC3168A069C9
:10707000C1F82405607D217D32680843C2F86C05A3
:10708000D4E900123068C0F80C15C0F81425207D32
:10709000012815D1A068411C02D0002104F093FC06
:1070A000E068411C05D08540C7F80855E06804F049
:1070B0009DFCD4E902123068C0F80825C0F810150C
:1070C000BDE8F08103F052BB2DE9F0470746008888
:1070D0008EB0804603F03EF8824604462D480025D7
:1070E0002A460178404600F069FD7879400734D59A
:1070F00001254FF6FF7603AB2A460721504606F0DE
:1071000035F9010004D0404607F03EFC00252BE095
:10711000B1463146049802F071FF064648450FD04B
:1071200004460146404602F0FFFF4046FFF7AAFD35
:1071300030B9404607F0FAFB4046FFF7A3FD48B1DF
:1071400022460721504606F087F9010003D0404649
:1071500007F01AFC00254E4506D0404606F0EAFA34
:1071600010B1504602F0E2FF02208DF81800ADF891
:107170001A807879400701D5012000E002208DF8BF
:1071800020008DF8215006A801F0CAFF0EB0BDE81E
:10719000F0870000142C00202DE9F0430546407CC8
:1071A00093B00E460024A0B107949DF81C0020F077
:1071B0000F00401C20F0F00010308DF81C00707B98
:1071C0008DF81D009DF81E0020F00600801C8DF833
:1071D0001E001C216846FFF770F99DF8000040F082
:1071E00002008DF80000697C11B140F0100001E050
:1071F00020F010008DF80000019403940494687C42
:1072000000B107A8CDE9050401278DF8427042F6C8
:107210001920ADF840000D94B07B8DF83400F07B60
:107220008DF835009DF83600142120F00600801CF2
:1072300020F019008DF83600307B8DF8440008A846
:10724000FFF73BF90DF140080DF13409ADF8287056
:1072500011A8CDE90889ADF82A40ADF82C700C9042
:10726000A888AB1D08AA6946AADF002838D1B068F3
:1072700098B38DF8427042F60810ADF840000D94B6
:10728000307C8DF834009DF8350020F0FF008DF83B
:1072900035009DF8360020F00600801C20F0190013
:1072A0008DF836000EA8B16800F0E0FF0646142104
:1072B00008A8FFF702F9ADF828600EA8CDE9088903
:1072C000ADF82A40ADF82C600C90E88805F10E026C
:1072D00008A9ABDF002803D101E0FFE7EC81002023
:1072E00013B0BDE8F083000010B50E490E4807F05A
:1072F000C2FBC1B20B484FF6FE72EC3800F00EFB39
:1073000000280DD008280BD0132809D0112807D049
:1073100043F20141884203D0BDE81040FFF744BD6D
:1073200010BD0000C42F0020982B00200A46014603
:107330001046AEDF70472DE9FC470025178806464A
:10734000158090F82D001446894630B13A46214602
:10735000484600F05DFC051E09D1B0784FF00C0ADC
:1073600018B32088C846001DB84202D95046BDE86F
:10737000FC87684679DF0028F9D12088032108F8C6
:10738000001020881921401C80B2208008F80010CD
:107390002088401C80B2208000EB0801BDF800006E
:1073A00008F080FA218808442080F0780222C8B1D1
:1073B000218896F9033001F1030C4846BC45D5D825
:1073C000425421884FF0010C491C89B2218000F8F9
:1073D00001C02188491C89B2218009F80130208828
:1073E000401C20807068B8B1218890F9003001F10C
:1073F000030C4846BC45B9D8425421880A22491C8E
:1074000089B2218042542188491C89B2218009F81F
:1074100001302088401C2080308950B1CDE90047E0
:107420004B460622022106F1080008F025FB051E46
:107430009DD1308A50B1CDE900474B460722032148
:1074400006F1100008F018FB051E90D1308B50B1EA
:10745000CDE900474B461522142106F1180008F02B
:107460000BFB051E83D1306A30B13B4622464946AC
:1074700001F077FB051EDBD1706A30B13B46224636
:10748000494603F0E1FA051ED2D196F82C0038B136
:107490003B4622464946304607F08CFB051EC7D1C5
:1074A000307838B13B4622464946304603F052FB1D
:1074B000051EBDD128465AE718B504460020ADF890
:1074C000000013466A46204600F006F8002802D065
:1074D000BDF80000204418BD70B588B182B1002409
:1074E000158803E0065D641C3444A4B2A54203D8A9
:1074F000061976789E4201D08C42F3D38C4201D398
:10750000002070BDA11C1180005D401E80B270BDC6
:1075100080F8301070472DE9F0410D00044606D088
:107520002CB195F87A000026012803D006E00E2041
:10753000BDE8F08195F89800012829D0D5F8A00081
:10754000042825D0D5F89C00042821D04FF001084C
:10755000A6702C2205F17801201DFEF787FF84F824
:107560003060D5F8A4006063D5F8A800A0634FF69A
:10757000FF70A4F8A80004F19400C4F8A400C4F8B3
:10758000AA60A4F8AE6084F8B060207810B104E07E
:107590000720CDE7FF2084F8540004F155011F2790
:1075A000C4F89410A4F8987004F198022846FFF7E4
:1075B000C2FE0028BCD115F13C0F0ED004F17401BD
:1075C000C4F89C10A4F8A07004F1A00205F13C00DE
:1075D000FFF7B1FE0028ABD103E0C4F89C60A4F82B
:1075E000A06084F85180208BA4F8480084F83C8087
:1075F000266484F8506060696064454604F13C028A
:10760000002104F1540072DF002891D125708FE72A
:1076100010B50288102A1BD0112A20D0262A1DD18D
:10762000007A0C46012801D0022817D1A078052144
:10763000401CB0FBF1F201FB1201204600F052F8B1
:1076400000280BD0A16B002908D0BDE810400847E6
:10765000C27B012A02D18088A1F8A80010BD0C4687
:10766000002184F8B2108088B4F8A8108842F5D1BF
:1076700020790028F2D10121DFE710B50C4602285D
:1076800001D0032810D1607800280DD00020607050
:10769000A178204600F026F8002805D0A16B00292B
:1076A00002D0BDE81040084710BD10B5044690F860
:1076B000540074DF012084F8B200002084F8B40084
:1076C00084F850000621204601F032FF002808D13E
:1076D000A178204600F006F810B1A16B01B18847EF
:1076E000002010BD2DE9F05F044600780F4638B148
:1076F000A770002003F084FF012620B1667007E127
:107700000820BDE8F09F0025C4F8AA50A4F8AE50A8
:1077100084F8B050A07910B1A078012806D0E079A3
:1077200068B1A078012801D0022808D1616B21B18D
:1077300084F8B1600820884701E084F8B15004F172
:10774000AB0100200A5C0AB1304603E0401C062869
:10775000F8D300204FF002084FF0030B012F06D0A2
:10776000022F0CD0032F0FD0042F15D110E0A179D8
:1077700029B194F8241011B908B130460DE0E1792F
:1077800011B108B1404608E0207A08B1584604E03B
:10779000607A08B1042000E02846A070616B41B116
:1077A000032801D0042804D1607910B194F8B20004
:1077B000A0B184F8B35004F13C0018210746FEF74D
:1077C0007CFE04F12C0084F83C60814606F0E6F86B
:1077D00058B194F82C0084F8510008E084F8B450B3
:1077E00084F8B36007208847E5E784F8516094F88F
:1077F000240050B1484606F0D1F820B194F8280092
:1078000084F8520001E084F8526084F85050A27865
:1078100004F1AA0104F194094FF0060A052A60D286
:10782000DFE802F078030F223F0084F83160C4F8EB
:10783000A450C4E9101584F83C808020A4F84800C6
:1078400051E084F8318094F82420384612B10722A0
:10785000027001E080F800B0228A8281C4F8A4504E
:107860004160E168B9603EE06069B860208BB88132
:1078700094F824003D4610B184F83CA001E084F85F
:107880003C60204608F0BCF840B185F81480042123
:10789000204601F04DFE20BB05211EE084F831B0EA
:1078A0001DE0E069B860208CB88194F824003D4662
:1078B00010B184F83CA001E084F83C60204608F058
:1078C0009FF848B185F814800421204601F030FE6D
:1078D00038B984F831A002E0042184F83110C4F8EA
:1078E000A490A07878B13A4604F15400D4F8A410DA
:1078F00072DF00287FF405AF94F8301094F854003C
:1079000073DF0028F6D1616B11B194F8310088471C
:107910000020F6E684F83150F5E70000F7B594B0A2
:10792000174605003CD0287C9DF85410002488425E
:1079300052D000264FF0010E0D9615A8ADF834E098
:107940000E90ADF83660E9880DAA4FF6FF70ACDFF7
:10795000040026D19DF854002874687CA0B30F96CB
:10796000109611961296E888ADF83C00BDF83600E6
:10797000ADF840000DA811900E981290A7F57F4029
:107980008DF83EE0FE3805D039460FA8FFF7CEFC53
:10799000044621E0684600F09DF800256F460FE0A0
:1079A0000E2017B0F0BD00BF07EB4506B08800F011
:1079B000CFF8022803D144B10FA9B088AEDF6D1C07
:1079C0000098A842F0D807E005E0B1880FA8FFF7BB
:1079D000ADFC0446F3E708242046E2E738B50D463F
:1079E000040018D0BDB12868206028796074FF2099
:1079F000207401208DF8020041F60F00ADF8000060
:107A0000221D69460120A8DF002803D1294620460F
:107A1000FFF7C2FB38BD0E2038BD38B5002924D091
:107A2000002822D00288502A1FD10546487C0C46E7
:107A300000281AD0E9886289A81D914215D1418990
:107A4000022912D1216800290FD00C3000F00AFC65
:107A500008B1002000E001208DF80000A888ADF8F2
:107A60000200226869462046904738BD70B5040080
:107A700012D001461C221448FEF7F8FC1248134DA0
:107A80000560206850B17ADF002806D120680168BF
:107A900029604068686005E00E2070BD0B487BDF00
:107AA0000028FAD108484FF6FF711438084A20F828
:107AB000041B0549343901600021FFF781F90028D2
:107AC000EBD0032070BD000094300020D42B0020A8
:107AD00099F902000149496801F024B8B03000204A
:107AE00010B5044600F08AF8002805D02146BDE80C
:107AF0001040024803F051B910BD0000C030002012
:107B000070B515460E46044607F086FF002809D0DA
:107B1000054800EB840080692A463146BDE8704084
:107B200001F044BD70BD0000B030002070B50546C6
:107B3000002400F063F838B12946044803F02DF919
:107B400008B1022400E00124204670BDBC300020B2
:107B500070B50546002400F051F838B129460448B4
:107B600003F01BF908B1022400E00124204670BD97
:107B7000B830002010B51821034803F0E9F81828A0
:107B800000D0C0B210BD0000B030002070B5054676
:107B90000C46084607F040FF60B1284600F02EF87A
:107BA00040B10548294600EB8400BDE8704018301C
:107BB00003F0F3B8002070BDB030002070B505466A
:107BC00014460E46084607F027FF002812D0284624
:107BD00000F014F800280DD00748294600EB860075
:107BE00018301CB1BDE8704003F0E2B8BDE8704049
:107BF00003F093B870BD0000B0300020142801D30A
:107C0000002070470146014803F0C7B8B430002097
:107C10007CB5054608880C460930904201D90C20F5
:107C20007CBD68466DDF0028FAD1218808206854A1
:107C300020881B21401C80B2208029542088401CB1
:107C400080B220802844DDF801100160BDF80510E5
:107C500081802088801D80B220809DF80010490816
:107C600000D0012129542088401C208000207CBDA8
:107C70007FB5044601208DF8060041F60A00ADF8F4
:107C80000400454A01A90120A8DF00287ED12288EE
:107C900004F13C0552B140482B46801C009042F64E
:107CA0002920616800F05AFE002873D1228952B160
:107CB00039482B460A30009042F62420E16800F053
:107CC0004DFE002866D1228A52B133482B4612302D
:107CD000009042F62520616900F040FE002859D14D
:107CE000228B52B12C482B461A30009042F62720A6
:107CF000E16900F033FE00284CD1228C52B12648B5
:107D00002B462230009042F62620616A00F026FEC3
:107D100000283FD1228D52B11F482B462A300090B7
:107D200042F62820E16A00F019FE002832D1216BCA
:107D300071B102A807F0E6FA17482B4632300090DE
:107D4000082202A942F6232000F008FE002821D1D3
:107D5000606B58B110492B463A31009102790168A5
:107D600042F62A2000F0FAFD002813D1A16B81B160
:107D700002A806F0F8F808482B4642300090072287
:107D800002A942F6502000F0E9FD00E002E00028E0
:107D900000D1002004B070BD322C002038B502881C
:107DA0000446212A2FD012DC1E484FF003011E4D3D
:107DB0000088102A01EB004011D0112A06D1227A46
:107DC0001AA104F04BF84FF6FF70688038BD3B2ACB
:107DD00023D0562AFAD18088132176DF0DE01AA12C
:107DE00004F038F8072000F0E3FB08B1FEF7DCFFF1
:107DF000A1886980174803F033F90028E6D0BDE870
:107E00003840FEF7D1BF00200090A08869468FDF80
:107E10000028DBD0FEF7C8FF38BD8088132176DF4D
:107E2000EBE70000F82D0020902B002044697363DD
:107E30006F6E6E65637465642C20726561736F6E1E
:107E40002025642E00000000436F6E6E656374652C
:107E5000642E0000002F002010B51A4C01886068C5
:107E600010290ED011292BD1401E606028D1FEF7B9
:107E70009DFE002824D02168002921D0BDE81040B3
:107E80000847D0B900210122084600F06FFB08B175
:107E900007280FD107220221012000F067FB08B15B
:107EA000072807D104220221002000F05FFB20B147
:107EB000072802D0216801B188476068401C6060D3
:107EC00010BD0000CC2B00202DE9F04701883B4E6F
:107ED00040F2F3194FF6FF7510291BD011293ED03F
:107EE000122954D0502946D1C188F289841D91426B
:107EF00041D1618902293ED18688304602F0D6F907
:107F0000050038D004F10C0000F0ACF9A8B3294604
:107F100030464EE0C17B8788044601292BD1A84614
:107F2000284602F0C3F9050017D02F8000202872E0
:107F3000234843464A460168C5F80A104068C5F818
:107F40000E0004F1100105F10A0002F07BFA6872DC
:107F5000F08900280FD129462AE0042013E0808808
:107F600002F0A4F9040006D06068FEF7A9FF08B18A
:107F700006F0EEFC2580BDE8F087FFE76868FEF7B5
:107F80009FFF0028F7D0BDE8F04706F0E1BC8788E6
:107F90000646384602F08AF90400ECD02B464A46E1
:107FA00006F1080104F10A0002F04CFA6072214661
:107FB0003846BDE8F04700F01BBE000094300020BA
:107FC000D42B00202DE9F04F0746858802883D48D4
:107FD000012197B08346102A09D0112A49D01A2AC4
:107FE0006CD1387AB1EB101F45D2012244E0354CF8
:107FF000083CA068C0430B9061680BA802F0F1FE3A
:108000000B990CA800F08EFD2C220CA96846FEF7F7
:108010002DFA0026E946A04610E000BF09EB460015
:108020005FF00004B0F804A008EB84005146001D86
:1080300002F073FE641C1D2CF6D3761C0098B0422F
:10804000ECD8142D05D317B00420BDE8F04FFEF78F
:10805000ABBE2946584602F0ABFE294608F10400A3
:1080600002F0A6FEF87B012828D016482946001DFC
:1080700015E029461AE000220221B1EB101F01D2BF
:10808000012600E000260F49083901F11000041D07
:10809000294682B102F08CFE36B12946204617B03F
:1080A000BDE8F04F02F084BE2946204617B0BDE877
:1080B000F04F02F032BE02F030FEF5E717B0BDE837
:1080C000F08F0000B830002010B504460748007853
:1080D00000280AD0204601F017FF204606F070FE67
:1080E0002046BDE8104001F0D7BB10BD042C002095
:1080F00030B50446008CC3B0A0F57F42FF3A23D0D0
:108100006A46204601F078FE0546ADF8F4000020EE
:108110003E903F90409041902189ADF8F8100121A8
:10812000ADF8FC008DF8FA103DA84090CDF804D1D0
:10813000208C3EA9AEDF002804D1BDF8F410A9427E
:1081400000D00C2043B030BD0820FBE738B5044612
:1081500008682060087960714FF6FF702084002065
:1081600084F82200A4F84C00F42084F84E0001208A
:108170008DF8020041F60D000D46ADF80000A21D7D
:1081800069460120A8DF00280ED12946204601F0CB
:10819000D1FD002808D1A86828B12946204600F062
:1081A0006BF8002800D1002038BD38B50288102AAD
:1081B00015D0112A15D0502A16D130F8062F8B89E8
:1081C0009A4211D10C46418902290DD1216800291A
:1081D0000AD00C3000F046F838B1002006E0808864
:1081E00001E04FF6FF70088438BD01208DF80000D3
:1081F000226869462046904738BD028C4B889A42D7
:1082000008D10A88A2F52063773B03D10979C91EFA
:1082100080F84E10704770B50446B0F84C000D461B
:1082200014280AD104F126012622881EFEF71EF921
:10823000B4F84C00401EA4F84C00B4F84C0004EB19
:108240004001401CA4F84C008D8470BD80F82210C1
:10825000704770B504460D460846FEF739F9208090
:10826000656070BD007800F0010070470A78027008
:108270004978417002207047F0B58FB00D46064630
:108280001C216846FEF719F900249DF800000394AC
:1082900040F002008DF80000012701948DF836703F
:1082A00042F63820049405940694ADF834000C94FA
:1082B000E87B8DF83000287C8DF831009DF8320085
:1082C000142120F00600801C20F019008DF83200E7
:1082D00007A8FEF7F2F80DA807900CA8ADF82470D7
:1082E0000890ADF82640ADF82870A8680B90F0888B
:1082F00006F1100307AA6946AADF0FB0F0BD00001F
:108300000149085C7047000088FF02000649095CCB
:108310004FF0A040D0F81005C84010F0010000D088
:10832000012080F00100704788FF02002DE9FC4128
:108330000646C0074FF000050ED0104F0024012262
:10834000385D009500231146019503F0D9FA641CAD
:10835000042CF4D300F046F8B0070DD5074E0024E6
:10836000361D0022305D032300951146019503F070
:10837000C7FA641C042CF4D3BDE8FC8184FF02001E
:1083800007490B5C4FF0A041D1F80425012098402B
:1083900020EA0203C1F808351040C1F80C05704707
:1083A00084FF02000249085C012103F03ABB00008F
:1083B00084FF02000249085C002103F032BB000088
:1083C00084FF02000649095C4FF0A040D0F8040584
:1083D000C84010F0010000D0012080F0010070477B
:1083E00084FF020010B500242046FFF7DBFF641C69
:1083F000042CF9D310BD10B500242046FFF7DAFF96
:10840000641C042CF9D310BD10B50246064B4FF086
:10841000FF3000215C5C944201D1084610BD491C2C
:108420000429F7D310BD000088FF020070B50C4E80
:108430000C004FF0000530600BD0012000F06AF80E
:1084400008B1022004E0002000F064F800B10B2025
:108450002070706810B9FEF7A9FB0546284670BD6C
:10846000CC2B002010B5002000F0D4F908B106286C
:1084700006D1012000F0CEF908B1062800D1002075
:1084800010BD00002DE9F0470D468146FFF7BCFF07
:108490000446042836D2DFF874801B481C4EA8F12D
:1084A0000C0725B3012D0ED0022D2BD104EB440077
:1084B00030444578002D25D0B968002922D02846BF
:1084C000BDE8F047084704EB4401755C0E44717841
:1084D00049B10E4A4FF40041093A8068FEF7ACFCFE
:1084E00008B987F80390B17808F80410E2E78068CB
:1084F000FEF7E6FC04EB4401314418F804008D78E3
:10850000A842D7D0BDE8F0878CFF0200C82B00201E
:1085100034300020042801D2FFF7F8BE0020704755
:108520000146104810B54088042907D007290ED00D
:108530000A2915D1BDE8104006F02EBC132176DFC4
:108540000CE000280CD0BDE81040FEF72DBCA0F5D3
:108550007F41FF3904D10448FFF7A7F80828F0D17C
:1085600010BD0000902B00200C2F002070B50023C0
:10857000042810D20D4D00EB4004012A02D101293C
:108580000CD00022094E00EB4000304461B10129BB
:1085900006D0022906D00723184670BD0E30C2B29D
:1085A0002A55F9E74270F7E78270F5E7343000208A
:1085B000044A014600201279D20702D0084600F092
:1085C0004DB87047BC2B002070B506461E480024ED
:1085D000C0E90161B00720D50025012211462846D7
:1085E000FFF7C4FF6D1C0446042D02D2002CF4D00A
:1085F00013E094B940F2666204211448FEF75AFB76
:1086000004000AD1FEF744FB040006D10F48104ACB
:108610000021001FFEF7D4FB0446F00712D0012012
:10862000FFF784FE74B909480A4A00210C38FEF7A6
:10863000C7FB040006D10548074A01210838FEF7A8
:10864000BFFB0446204670BDBC2B002098FF0200F3
:10865000E1880200D9A402007F6C02002DE9F05FDE
:108660006A4C054600266078B34618B184F801B01C
:1086700001F01AFF664F4FF47A694FF4C87A4FF051
:108680000108182D62D2DFE805F0AC0C0C31404D2A
:1086900062676B746B74BE7D7D7D7D7DACAFB2B562
:1086A000BEBE0020FFF78EFE00284FF0000008D06D
:1086B000FFF778FE022D02D14FF4E16008E0484652
:1086C00006E0FFF777FE022D01D1C82000E05046FA
:1086D000410CC0034FF4FA72801841F1000125707B
:1086E00052000023FDF77EFE01462AE00020FFF73E
:1086F00069FE00284FF0000004D0FFF753FE4FF44E
:108700004870E5E7FFF756FEDFE70020FFF75AFE67
:1087100000284FF0000002D0FFF744FECFE7FFF73C
:1087200049FED4E70020FFF74DFE00284FF000007F
:1087300002D0FFF737FE01E0FFF73CFE257041F65F
:108740009A1100223868FEF777FB064646E00020C3
:10875000FFF716FE257008E0002051E025703DE08F
:1087600084F801800120FFF70BFE002240F6CD4186
:10877000E8E784F801800120FFF702FE00224FF4B1
:108780008041DFE77868FEF79BFB0646D5F11100D4
:1087900000D02EB10220FFF705FE84F802B01DE0E4
:1087A000012816D980B2C8214843C117C90341EA3C
:1087B0005041C0034FF4FA72801841F10001520099
:1087C0000023FDF70FFE014600227868FEF734FB18
:1087D00006460220FFF7EEFD84F802803046BDE831
:1087E000F09F01F061FEB9E701F05EFEB4E701F031
:1087F0005BFE04E001F058FE0020FFF7DBFD0120E6
:10880000FFF7D8FDAAE7FFF7F6FDA7E7BC2B00208E
:108810008CFF0200012107F096B900002DE9F84312
:108820000546861C00208DF8000090460F464FF04C
:1088300001096846FEF754FB1B4C20683860D4E9F8
:108840000001401AA16804F21C47081A0EE0012139
:10885000384602F0C0FA01F0DFFF0146384602F068
:10886000BAFAD4E90001401AA168081A401C8642ED
:10887000EDD8B8F1000F03D0052065F3891002E0B0
:10888000062065F39F50A2682168114004EB810126
:10889000C8602068304420609DF80000FEF744FB6B
:1088A0004846BDE8F88300000838002030B48268EC
:1088B0000468531C8360A154D0E901128A4202D398
:1088C00030BC02F0CABC30BC70470000034803C88B
:1088D000814201D1012070470020704708380020F4
:1088E00000780221FFF7CEBD05494FF0FF3208287E
:1088F00041F8202002D3084480F848207047000047
:1089000098330020F0B54FF0FF3512B10023082650
:1089100001E008230C260C4C05E000BF54F823703E
:108920007F1C04D05B1CB342F8D32846F0BD261848
:108930005DB286F8305044F82310002AF5D1E118D2
:1089400081F84800F1E7000098330020024908440C
:1089500090F9300070470000983300202DE9F04373
:108960008FB01E46DDF8589015460F00804602D1A4
:108970000020FEF719FA15B90020FEF715FA1C21A0
:108980006846FDF79AFD00249DF80000039440F02E
:1089900002008DF80000012001948DF83600049447
:1089A00005940694ADF834800C9430788DF830003E
:1089B00070788DF831009DF83200142120F0060007
:1089C000801C20F019008DF8320007A8FDF775FD16
:1089D0000DA807900CA808900748ADF82450ADF8F2
:1089E0002640ADF828500B974B4607AA69460088E9
:1089F000AADF0FB0BDE8F083322C002070B504462A
:108A00004FF6FF750A462846AC4208D14FF48074F1
:108A10002146104605F018F9A04209D070BDFF2C80
:108A2000FCD82146104605F002F908B1204670BD79
:108A3000284670BD70B5084C050009D01034216877
:108A4000002907D008682060496828468847F6E76B
:108A50000834F4E770BD000084330020054A01218A
:108A600020B1012805D19170FFF7E4BF51700020BB
:108A7000FAE77047843300202DE9F05F264841680B
:108A8000F1B3DFF898B00E688146DBF800408768E4
:108A90008078E11B21F07F45ED1CB0B9DFF88080C4
:108AA0004FF48030C8F84403C8F804031120FDF7E0
:108AB00023FE1120FDF72BFE4FF0010AC8F800A09D
:108AC0002F2003F05FFE89F802A0B54200D23546A0
:108AD000124BE8193C3320F07F401860DBF800109F
:108AE0005A46091B21F07F41001B20F07F40C91C22
:108AF00081420FD9106818602F2003F043FE00E078
:108B000004E0BDE8F05F1120FDF70CBEBDE8F05FAA
:108B100005F020BDBDE8F09FB82C002004150140F1
:108B20000010014073B58CB00646002000900D98EF
:108B300080B100246D4621460DA802F02EF930B117
:108B4000009805EB400084800098401C0090641C55
:108B5000142CF0D32C2269463046FDF787FC0EB06A
:108B600070BD2DE9F04117880646B81D14460D4624
:108B7000984202D90C20BDE8F081318807220629ED
:108B80000AD34FF4486C4FF6FF73614501D99942FF
:108B900002D17088062801D21046ECE7604501D961
:108BA0009842F9D1994203D0984201D08142F3D83A
:108BB0000520E85520881221401C80B220802954CD
:108BC0002088401C80B220804119308806F06AFE5F
:108BD0002188084480B220804119708806F062FE26
:108BE0002188084420800020C5E7FEF7DDB800009A
:108BF00038B54A7A0F4B62B100220A7259690029CE
:108C000006D001228DF80020ADF8020068468847A2
:108C100038BD0A7A62B19B684C6802461946204604
:108C2000FEF70AF90028F3D0BDE8384005F090BE01
:108C30005B68F1E794300020F0B585B016460F462A
:108C400004461D4614220B496846FDF70FFC0A48EE
:108C50008DF80870ADF80240ADF80A608DF80C5040
:108C6000017800222046FEF7A9FF684600F058FA76
:108C700005B0F0BDA4000300142C0020F0B587B0AF
:108C8000074600200490ADF810100590ADF81210C2
:108C90000190029001AA04A9384690DF060022D074
:108CA00003F016FD114C0346012520883A4605EBDA
:108CB00000400F4903F0D9F8BDF8042012B9BDF8FF
:108CC000060038B12088BDF8063005EB004009A148
:108CD00003F0CBF8BDF808202AB12088154905EB30
:108CE000004003F0BBF807B03046F0BDC42D0020B3
:108CF0006804030054686520726571756573746556
:108D0000642054582F5258207061636B6574206C36
:108D1000656E67746820697320746F6F206C6F6E66
:108D2000672062792025752F2575206F637465741F
:108D3000732E0000B404030030B5044685B0002152
:108D40001B4804F074FF00282FD00025204600F0B7
:108D500030FF68B1112812D086281BD0A0F54051F1
:108D6000023903D00146204605F0FAFD294607E006
:108D700005B029462046BDE8304001F02BBD012159
:108D8000204601F027FD05B00021BDE8304008482D
:108D900004F081BF142207496846FDF767FBADF870
:108DA0000240684600F098F9E0E705B030BD0000E9
:108DB000DD2B0020CCFF02007FB50C4610B1012056
:108DC00004B070BD2079002638B141F61D55012848
:108DD0001BD0022826D00F20F2E702202071029635
:108DE0000396E0680190694601A805F0CBFA50B1FE
:108DF00002988188E18000882081BDF800100298E7
:108E000005F03EFBDCE70A20DAE70A4B6A46002160
:108E1000A01D05F073FA38B1064918398E61CE618C
:108E20000A28CDD12846CBE702488188019805F071
:108E300027FBF5E7F82C00202DE9F0470025DFF8A7
:108E40008C803CE06068002100EBC5060120327890
:108E50009146FDF7F8FAD4E9062300EA020701EA91
:108E6000030C57EA0C0728D082438B434846C4E9D9
:108E7000062303F049FD3278824691460120002105
:108E8000FDF7E1FAD4E9042300EA020401EA03074A
:108E90004A4650460021FDF7D6FA44404F403C4335
:108EA0000BD17078012801D0012100E00021726807
:108EB00081EA0A010AB1484690476D1CEDB298F864
:108EC000000044468542BDD3BDE8F087982C0020C1
:108ED00010B50021024801F099FF80F3100010BD89
:108EE000243C00200E4910B50A784C780023A24299
:108EF00012D0521CD2B20A70022A00D10B70084A5A
:108F00000B780C3252F8232002608868104420F05D
:108F10007F408860012010BD0360002010BD00006C
:108F2000B82C002013460A460021FFF785BE00003A
:108F30002DE9F843104D0F4680461E46914669467E
:108F4000286801F0BEFE040014D01C21FDF7B5FA1C
:108F500001202071C4F81490380BC4F80080C4E9D3
:108F600002606946286801F0CDFE05F05BF900203B
:108F7000BDE8F8830420FBE78001030010B5037807
:108F80000022072B06D2DFE803F005040610202993
:108F900030000A7010BD01230B7003898B81838818
:108FA000CB81C06888600A7410BD02220A700289F1
:108FB0008A818288CA81C2688A60807D062802D040
:108FC0000020087410BD0120FBE703220A70C2884C
:108FD0008A810289CA81C068886010BD04230B7031
:108FE000C0888881CA818A6010BD0520087010BDC4
:108FF00070B5064D0646002455F8241009B13046D8
:109000008847641C042CF7D370BD0000883500200D
:1090100030B50446006887B00D46806800281FD030
:1090200018216846FDF749FA0195A0680590207956
:1090300010B1012810D107E001208DF8000020694F
:109040000290E068039005E002208DF80000E068DF
:109050000003029060690490206881686846884730
:1090600007B030BD70B586B015460C00064619D065
:10907000112C17D0082C15D014216846FDF71DFAC5
:10908000ADF80260304601F065F8ADF804000D2C33
:109090000AD0862C1CD007208DF800000294684668
:1090A00000F04CF806B070BD03208DF8000025B12B
:1090B0002878C00701D0012000E002208DF80800C8
:1090C00000208DF80C0041F20110ADF80A00E6E72F
:1090D00006208DF80000E2E710B50446408801F054
:1090E00039F8A080024801682046BDE810400847D2
:1090F000E42B00202DE9F04107460024064E074DE1
:1091000005E000BF56F8241038468847641CE8780C
:109110008442F7DBBDE8F08138330020042C0020C6
:1091200010B50446408801F015F8A0800248016897
:109130002046BDE81040084778000300014909684F
:1091400008470000CC0003007047000070B586B0EF
:10915000044614216846FDF7B0F9A0890125A0F561
:109160004040ADF8040020782A4E062833D2DFE8CC
:1091700000F0320303032C48A08900F0BDF930B998
:10918000E08943F6FE71A0F54040884223D8A07BD9
:109190008DF80800207803280FD000208DF80900F2
:1091A000A0680390606850B109208DF800006068E5
:1091B0000490684604F098F90DE00120EEE70820DD
:1091C0008DF800008DF81050F3E7A08900F094F9B5
:1091D00008B1E08930B17078002801D004F0B4FA09
:1091E00006B070BD606820B10B208DF8000075706E
:1091F000DFE70A208DF80000BDF8040004F02EFB24
:10920000F5E713208DF800004FF6FF70ADF804006D
:10921000CFE70000F42B002038B504460E48007854
:10922000A8B1A4F57F40FF380FD0684604F02CFFAA
:1092300078B10521017001210171C480684604F0F4
:1092400031FF04F0E1FF002038BD042038BD0220CA
:1092500038BD082038BD0000002D00200C4808B59E
:10926000007888B1684604F00FFF78B106210170DC
:10927000684604F017FF0748017809B1012101731E
:1092800004F0C2FF002008BD022008BD082008BD70
:10929000002D00204C360020F0B587B01421684620
:1092A000FDF70BF92B4C207818B16846FFF7A0FEAC
:1092B0004EE0201D01F08CFDB8BB4FF0102041693D
:1092C0000004026940694B1C01D100FB02F12248F5
:1092D00000220161A1F54051C160204902F04CF922
:1092E000002820D11F481C238C221D49006801F052
:1092F000D5FC03F0E9FE051E14D0022812D0002789
:109300000126062D12D005A804F0BEFE88B1067015
:109310000C2D18D2DFE805F0170F170F17161716C8
:10932000171113110B2007B0F0BD11E02670676014
:10933000BBE70820F7E7077105E0032100E0022101
:10934000017100E0067105A804F0ACFE04F05CFFBA
:109350000020E8E7002D0020B02D00209001030040
:1093600098350020F800030038B5040014D0694691
:1093700005F008F8A0B1BDF8000000EB8001094835
:1093800000EB8100C16849B1A17A39B1C168491EB9
:10939000C1600020A07238BD052038BD062038BD50
:1093A0000A2038BD243600201FB501A9684604F004
:1093B000A5FF04B010BD07B513460A466946002054
:1093C00004F09CFF0EBD07B513460A46002168460F
:1093D00004F094FF0EBD20B119B1006808600020B0
:1093E0007047052070470000F8B50D46040018D0FE
:1093F000BDB1694604F0C6FFA8B1BDF800000B4935
:1094000000EB800001EB800001210C30666801F068
:10941000E2FC2E6060680C3068600120A0720020C1
:10942000F8BD0520F8BD0A20F8BD00002436002054
:1094300018B10323002206F075BC052070470223F3
:10944000002206F06FBC12B1022306F06BBC0520AF
:1094500070470000084910B50A69042A0AD0074A73
:10946000096942F8210004480121103001F0B3FCE1
:10947000002010BD0C2010BDE02C002088350020FD
:1094800038B5044609480D46007858B164B16946BC
:10949000284606F041FD002803D1BDF800102180C8
:1094A000658038BD022038BD052038BD002D002064
:1094B00010B504460E48007898B1A4B1218802295D
:1094C00013D80C4A01EB810002EB800260885289BC
:1094D000C31C934209D806F013FD00202080608051
:1094E00010BD022010BD052010BD042010BD0000DD
:1094F000002D00202436002043F6FE71A0F54040E8
:10950000884201D8012070470020704710B50446FA
:109510000078182802D1FEF72DFB207010BD10B581
:1095200004460078182802D1FEF724FB207010BDF5
:1095300070B50D460446B0F89810D0F8940001229A
:10954000FDF7BAFF00B1057004F13C0204F194018B
:1095500004F1540072DF70BD70B513460022064658
:109560001546862902D0112902D002E0012200E02E
:1095700001250D4C73B1A179FEF720FB2A466179D4
:109580003046FEF71BFB0022A1783046FEF716FBA3
:10959000002203E0A178FEF711FB2A4661783046ED
:1095A000BDE87040FEF70ABB1C2C0020F7B517463B
:1095B0000E0011D00098002560B1002421466846B5
:1095C00001F0EBFB18B1A0B23946B0476D1C641C2A
:1095D000142CF3D32846FEBD0020FEBD406804F0E5
:1095E00073BD00000EB517A19DF8080020F00F0014
:1095F000401C20F0F00010308DF808000A2202A86C
:109600007CDF08B1FDF7D0FB40F2413078DF08B1D4
:10961000FDF7CAFB0020009001904FF4A071ADF857
:109620000400ADF800104FF4C8704FF40271ADF8AB
:109630000600ADF8021068467ADF002801D0FDF779
:10964000B3FB0EBD4E6F726469635F48524D0000FC
:1096500010B508880C46A0F52061773909D1084873
:109660000321A3880088628801EB004005A102F075
:10967000FCFB2146BDE810400E48FEF7BEBD0000D1
:10968000F82D00204741545420415454204D545546
:10969000206F6E20636F6E6E656374696F6E20302D
:1096A000782578206368616E67656420746F202573
:1096B000642E0000882E002070B508B1012070BD16
:1096C000194C0025207B08B1257301E000F0A0F8BB
:1096D0002078082826D2DFE800F02504080C1025A1
:1096E0001420BDE8704000F021B8BDE8704000F0E3
:1096F0007DB8BDE8704000F05FB8BDE8704000F094
:109700003BB86088084900EB8000283901EB8000F5
:109710004068BDE8704003F0B7BC6560BDE87040CC
:1097200003F0C0BC0F2070BD4C3600201149F0B4CE
:109730008A1C00200346A1F128050C18A67A4EB118
:10974000A37200EB800405EB8404E66816B9247C60
:10975000012C0AD0401C80B20228EED30B704B8043
:109760004B60F0BC41F61D5070471080F0BC00F01B
:109770003DB800004C3600200C48418801EB8102C6
:10978000A0F1280101EB8201CA6852B105210170E4
:10979000074802218180016800230122054801F069
:1097A00055BE042202704968F6E700004C360020DE
:1097B000082D0020B02D002038B50A4908480324A0
:1097C0000B684268898803EB810153880470DB1CB5
:1097D00000201B0400909B0B034801F0A7FF38BD3D
:1097E0004C360020082D0020B02D0020074910B570
:1097F0004888091D04F016FE18B1BDE81040FFF7B7
:10980000DBBFBDE81040FFF7B7BF00004C360020BB
:10981000F0B51F481F490125067802248B88A0F166
:109820002802082E19D2DFE806F00418181B222F90
:109830002F170189491C01810021418080F80C10FB
:1098400001EB810312F8233043B100234418491C73
:1098500089B2A3720229F3D30570F0BD0123F5E7A5
:1098600042685288D21C1A448A800470F0BD46882F
:109870000D6806EB860602EB860256680E605560A0
:1098800013818C80062100E007210170F0BD0000EB
:109890004C360020082D002030B501888488224DE8
:1098A00085B0502924D0522902D0542931D103E067
:1098B000204600F05BFF2CE014221C496846FCF7B0
:1098C000D5FDADF80240204600F044FCADF80400A0
:1098D00000F022F9002269792046FEF76FF9002294
:1098E00029792046FEF76AF96846FFF7F5FB10E094
:1098F000017B01290DD1817A01290AD10089A0F5C6
:109900002451023905D10121204600F063FF06F001
:1099100039F800220649E878FEF7F2F805B0BDE80C
:10992000304005F0D5B80000DC2B0020F4FF020029
:10993000C570020010B50446007800280FD1608879
:1099400000F014FF608800F081F9002807D0044976
:10995000608801220979BDE81040FEF72FB910BDDB
:10996000DC2B002010B5124C00202070FEF702F90D
:10997000A070FEF7FFF8E070FEF7FCF82071FEF72C
:10998000F9F86071A17818290FD0E17818290CD066
:109990002179182909D0182807D00121601C04F06A
:1099A0003FF901202070002010BD032010BD0000F1
:1099B000DC2B00207CB50446007808282FD1607A83
:1099C00038BB207A4FF6FF7501280DD0072802D04A
:1099D000082824D11EE0A08800F0FAFAA8421ED080
:1099E000012100F0F7FE1AE0A0886A46012103F089
:1099F00093FC70B90198007858B1A08800F0E8FA9B
:109A0000A8420CD0084901220979FEF7D7F805F0E1
:109A10005FF804E004480021401C04F03CF9BDE874
:109A20007C4005F0AFBF0000DC2B002010B50446E1
:109A30000A4841782046FEF7A9F868B10848002195
:109A400001EB410200EB82025288A24201D1C8B26E
:109A500010BD491C1429F3D3FF2010BDEE2B0020AC
:109A60002831002070B5094D094E002404EB440054
:109A700005EB800071784088FEF788F820B1641CFF
:109A8000142CF3D3FF2070BDE0B270BD283100204C
:109A9000EE2B00202DE9F0418046024601200021F6
:109AA000FCF7D1FC1A4F05460E467868FDF708FA18
:109AB00000280CD1174CD4E9062110462A4001EAAF
:109AC00006031A4305D0A843B143C4E90601BDE823
:109AD000F081404602F018FF30B1D4E90401284378
:109AE0003143C4E9040105E0D4E90410A943B043BB
:109AF000C4E90410D4E9060128433143C4E906014E
:109B0000A1687868BDE8F0410022FDF795B9000032
:109B1000DC000300982C00201CB5054AD2E9021293
:109B2000CDE900120022694603F01BFC1CBD0000B9
:109B30000C00030003484FF6FF7181800121017082
:109B400000207047E82B00202DE9FC41804600F002
:109B500001FB002403250127A0F57F412646FF399C
:109B600008D06A46082103F0D7FB18B90198841D74
:109B70008688056832462B4621464046B1DF0428D8
:109B800004D0082804D00B2808D002E0112000E0FF
:109B90000020002F00D10B20BDE8FC810027A80782
:109BA00001D50125E6E73443F5D0002426460325F8
:109BB000E0E72DE9FC41804600F0CCFA0646A0F52E
:109BC0007F40FF380ED001252A466D1C0027ADB21C
:109BD0006B460821304603F0C9FB040006D0072C71
:109BE00025D025E043F20200BDE8FC810199032362
:109BF0000A1D0B604046891DB2DF040004D00C2C06
:109C000009D0052C09D009E032460821104603F09E
:109C100023FC04460CE0012700E000240821304624
:109C200003F006FC00B10324002FCDD100E00C248A
:109C30002046D9E704488088A0F57F41FF3901D04C
:109C400004F050BF70470000E82B00200EB502A9B9
:109C5000019100F07FFA6A46012103F05DFB08B133
:109C600000200EBD019800780EBD00002DE9F041E6
:109C700007464FF6FF760A48B3DF10B10320BDE870
:109C8000F081074C43F20305A41E32466188384632
:109C9000AFDFA842F3D16088401C6080F5E7000088
:109CA000EA2B0020428800EB82020C328A4201D962
:109CB000022070478188A1F57F42FF3A03D00088D7
:109CC00008B10020704701207047884204D2006824
:109CD000401C01D0012070470020704710B5124988
:109CE000124804F0C8FE114C81B2103C6068401C60
:109CF00060600F48FEF7FCF958B1082809D0132816
:109D000007D0112805D043F20141884201D0FDF768
:109D10004BF860680321B0FBF1F201FB120000B1C7
:109D20000120207010BD0000D42F0020A02B0020A7
:109D3000882E002070B5CCB00024054644949DF8D0
:109D400010010E4620F00F00401C20F0F0001030F3
:109D50008DF81001087B8DF811019DF812011C216E
:109D600020F00600801C8DF812013DA8FCF7A5FB31
:109D70009DF8F4003E9440F010008DF8F40044A8E3
:109D80004094CDE9414001208DF82E0142F6372064
:109D90004394ADF82C014A94707B8DF82801B07B78
:109DA0008DF829019DF82A01142120F00600801C5D
:109DB00020F0180040F001008DF82A0145A8FCF7BA
:109DC0007CFB4BA845904AA846906A46002128464D
:109DD00000F012F8ADF81C01F420ADF81E41ADF80A
:109DE0002001CDF824D1E88805F1080345AA3DA952
:109DF000AADF4CB070BD00002DE9F0410446407967
:109E00009046002500B1042594F8220008B145F0E1
:109E10000205CAB2FF2908D9090A88F8012045F0CD
:109E2000010588F80210032602E088F801200226C6
:109E3000B4F84C0008B145F0100500271BE000BF46
:109E400094F84E10B21C91420BD2B4F84C0004EBC3
:109E50004701C01B420004F124002431FCF706FB3B
:109E60000DE004EB470008EB0601808C0870000A47
:109E70004870D6B27F1CB4F84C00B842E0DC34F82D
:109E80004C0FC01B208088F800503046BDE8F081A0
:109E90003EB5027802230C46B3EB520F17D1B0F84F
:109EA0000110ADF80010C1788DF802108188ADF86E
:109EB000041080798DF8060002AA01A92046FCF75B
:109EC000B5FE032202A96846FCF709FB08B1002091
:109ED0003EBD01203EBD000010B50C46FFF7A6FDBB
:109EE000FF280CD0074900EB400001EB80004168DF
:109EF00021600189A180807AA071002010BD052019
:109F000010BD00002831002070B5018890B01029E4
:109F100059D1011D2C226846FCF7A8FA9DF80400CF
:109F20004FF6FF76032134466D46B1EB500F2AD031
:109F300003F048FB9DF8040040080ED001280CD027
:109F4000022820D118E00D99281D1131FCF709FED7
:109F500018B100BFBDF82C4015E00CAA0BA90720D2
:109F600003F004FB0028EED10DE00D99281D491CDB
:109F7000FFF78EFF0028EDD10CAA0BA9072003F0F4
:109F8000F5FA0028F1D1BDF80000291D00F030FEDF
:109F9000B44218D0BDF80000214600F0C5F8BDF865
:109FA0000000ADF82E000020ADF83040074E8DF8CF
:109FB0002C000BAD044600BF56F8241028468847F5
:109FC000641C022CF8D310B070BD00002000030008
:109FD000094A002101EB410332F82330834205D1C5
:109FE00001EB410002EB800040887047491C1429B6
:109FF000F0D34FF6FF707047283100203EB50C4675
:10A00000054603F0DFFA0BE0BDF80000A04207D0E0
:10A010002846029900F02EF810B1BDF800003EBDB0
:10A0200001AA6946072003F0A1FA0028ECD14FF6F7
:10A03000FF703EBD10B50D4C18200D4A6070002019
:10A040004FF6FF7100EB400302EB8303401C598085
:10A050001428F7D3FDF78EFD6070182803D0012077
:10A060002070002010BD032010BD0000EE2B00204A
:10A07000283100202DE9F0410C46054600F111077A
:10A0800001F111061022491C401CFCF728FA48B9BE
:10A09000681C00F0F9F928B1601C00F0F5F908B16E
:10A0A000012400E0002431463846FCF75AFD3B7895
:10A0B0000222B2EB530F0CD00321B1EB530F08D0A7
:10A0C0003378B2EB530F04D0B1EB530F01D0012121
:10A0D00000E00021084201D18C4302D00120BDE8FC
:10A0E000F0810020FBE7018811B9421892780AB18B
:10A0F00001207047491C0829F7D30020704710B58C
:10A100000C460346FFF7EFFF00280AD01888218885
:10A11000884205D10822A11C981CFCF7E0F908B17F
:10A12000002010BD012010BD03F0ECBB70B504464B
:10A13000FFF74EFF0546204603F0F1F84FF6FF719A
:10A1400004468D4203D014B9284603F0DBFB2046B9
:10A1500070BD000010B5FFF769FCFF2805D0044969
:10A1600000EB400031F8200010BD4FF6FF7010BD2D
:10A17000283100203EB5044603F024FA0EE0019990
:10A1800020464631FFF7BBFF28B9019920462A3106
:10A19000FFF7B5FF10B1BDF808003EBD6A4602A941
:10A1A000072003F0E3F90028E9D14FF6FF703EBD28
:10A1B00010B50A4941600A4800F00AFE58B902F099
:10A1C00011FA07491C238C22087404488C39001F9B
:10A1D000006800F063FD002010BD00008401030052
:10A1E000E83600202DE9F0412D4F002518B17D60A3
:10A1F0000120BDE8F0810879012258B1294E0128DB
:10A200000CD0274C4FF002080834022821D0032834
:10A2100042D128E00A7102F045FF3BE05FF0000008
:10A2200000EB800116F82110022908D0401C80B2F2
:10A230000228F5D33A707D6041F61D50D9E700EB56
:10A24000800006F8205006EB8000406802F01CFFFA
:10A2500020E00D71A4F80480002301221248216837
:10A2600001F0F4F816E00D71206802F00DFF0D49C1
:10A2700023682831498801EB810206EB8201D1F87D
:10A2800004C0C4F800C04B60A3880B81A4F804800C
:10A2900006F822500028ACD07D600E20A9E700000F
:10A2A000002D002024360020B02D00200146034858
:10A2B00002888A4200D000207047000080300020D1
:10A2C0002DE9FC5F0E008346DDE90C47C6F1000076
:10A2D00098469246814600D40846012503E000BF17
:10A2E00090FBFAF06D1C5045FADAA84500D94546B6
:10A2F00024B1002E01DB780700D5641EB80702D513
:10A30000B8F1000F0AD0F80708D13CB1A54205D238
:10A3100020215846641EFEF7C9FAF6E7002E02DA3D
:10A320004E462D2102E0780703D52B215846FEF733
:10A33000BDFA07F0030002280BD1B8F1000F08D1D5
:10A340003CB1A54205D230215846641EFEF7AEFA54
:10A35000F6E7CDE90047434652463146584605F0F8
:10A36000B7FABDE8FC9F000070B50D4604460068D2
:10A370004FF4887102F0CCF94FF49071206802F02C
:10A38000C7F94FF49271206802F0C2F94FF4A2713C
:10A39000206802F0BDF920681249C0F80413206853
:10A3A0006907000B40B2090E002806DA00F00F0022
:10A3B00000F1E02080F8141D03E000F1E02080F8B7
:10A3C000001420680121000B40B200F01F029140F0
:10A3D0004009800000F1E020C0F88012C0F80011B0
:10A3E00070BD0000100302000246002012689307AF
:10A3F00002D0530702D47047500714D502F003006F
:10A40000012802D002280CD105E0C2F383100B68AA
:10A41000801C184404E00223086803EB92521044A5
:10A42000086001207047086800EB9253C2F389105E
:10A43000401CEEE70248007A002800D00120704757
:10A44000E8360020F0B58488A518944200D822464A
:10A45000A41AC288D6189A4200D81346D21A4B883A
:10A460000788BB420CD34088834209D88888A04221
:10A4700006D3A84204D8C888904201D3B04201D97B
:10A480000020F0BD0120F0BD0021425C0AB1012096
:10A490007047491C1029F8D300207047800701D06D
:10A4A00000207047012070470A4810B5807860B1DD
:10A4B000002401E0022C06D02046FDF773FF641C47
:10A4C000042CF7D310BD0324F6E7BDE81040FDF7D8
:10A4D00089BF0000BC2B002003480179C90702D0C6
:10A4E0000078FEF7BBB87047BC2B0020F721018035
:10A4F00017214180002101714171FB2181711B21D4
:10A50000C17170472DE9FE4F2B4D984691460F00C3
:10A51000824601D000260DE0684600F095FB6A46B1
:10A520000021504602F067FE2878009E10B99DF881
:10A53000090098B14A463146504604F09DFD044654
:10A54000014600225046FFF707F80D2C32D008DCF8
:10A5500084B3082C2ED00B2C0BD12BE00520BDE8AA
:10A56000FE8F112C10D0862C1AD0A4F54050023842
:10A5700020D00325B8F1000F04D0324621465046C2
:10A58000FEF770FD2846EAE73A4629795046FDF77E
:10A5900015FB4A46E9785046FDF710FB0025E9E730
:10A5A0003A4629795046FDF709FB4A46E978504674
:10A5B000FDF704FB2546DDE71C2C00202DE9F041CA
:10A5C000204F0E46154604463978FDF7DFFA00287D
:10A5D00035D0204602F006FE50B32046FFF7BAFD04
:10A5E00080462046B978FDF7D1FA08B1012700E08E
:10A5F0000227204603F09EF80028404602D0FFF7CD
:10A6000095FD0DE0A8F57F41FF3909D0072102F043
:10A610000FFF010004D0052902D0204604F0B4F950
:10A620002B46324639462046BDE8F041FEF704BBD2
:10A630002A4631462046BDE8F041FEF773BCBDE82E
:10A64000F0810000142C002070B5094D0646E97811
:10A65000FDF79CFA044629793046FDF797FA014642
:10A6600022463046BDE870400123FFF74BBF000093
:10A670001C2C00202DE9F047394E002780463D462E
:10A68000DFF8E090D6F804A057E003D00446D0F8F5
:10A690001C8035E099F8002002EB4201521CD2B236
:10A6A00089F8002009EBC10199F80230091D9A428E
:10A6B00001D189F8005048680A780446012A12D06E
:10A6C000022A02D0032A3BD108E004F09BFE00B12D
:10A6D0000127257434E00574C06900E07068002823
:10A6E000F9D170602CE0207C50BB88686060C8683D
:10A6F000A0600869E0604869A061F07800B1656019
:10A700006268B168184B501A20F07F40984202D21C
:10A71000A168084406E0881AA16820F07F408142C1
:10A7200002D9081A206000E0256065600120A5605C
:10A7300020742046E56104F047FEB8F10000A4D182
:10A7400099F8001099F801008142A3D117B97168F6
:10A75000514502D00120BDE8F0870020FBE7000052
:10A76000B82C002064340020FFFF7F0030B585B096
:10A770000546002414216846FBF79FFEA5F57F409F
:10A78000ADF80250FF3815D02846FFF7DDF998B133
:10A790000B2815D0112811D0A0F54051023903D053
:10A7A0000146284604F0DCF809482246C1782846CC
:10A7B000FDF704FA05B030BD0E2002E00124F3E7F6
:10A7C0000F208DF800006846FEF786FCECE70000DD
:10A7D000DC2B00200A4602498978FDF7EFB900001A
:10A7E000DC2B0020F8B5054600780C4600262042F8
:10A7F0000FD100208DF800006846FCF771FB287827
:10A80000204202D12043287001269DF80000FCF769
:10A810008BFB3046F8BD00002DE9FF4100262348A0
:10A8200000F0D3FA2148001F074600F0CEFA204C72
:10A8300060680090A56800E000986946284004EB35
:10A8400080000C30FFF7D0FD0028F5D101AA009957
:10A8500001EA050304EB8303491CDB6842F820305E
:10A86000401C00910228F2D3019800F00300012857
:10A870000BD0022810D10198032101EB90500099D0
:10A88000BDF80A6001EB900005E00198BDF80A6090
:10A89000C0F3831008440090384600F093FA08B1E2
:10A8A0000098606004B03046BDE8F081203C002094
:10A8B00008380020ACB04FF40041002001F03CFB10
:10A8C00008B1FCF771FA01F0A7F904F029FE4D492F
:10A8D0000320FDF779FE08B1FCF766FA694600200F
:10A8E000FDF7A4FD08B1FCF75FFA9DF8000002280F
:10A8F00074D0002601F03EFC08B1FCF755FA01F0D7
:10A9000017FE08B1FCF750FA0024694601200094B4
:10A9100001F072FC08B1FCF747FA684601F018FD37
:10A9200008B1FCF741FAFEF75DFE3749374800F001
:10A93000E2FA08B1FCF738FAAC216846FBF7BDFD36
:10A9400002208DF8000001208DF802000621032569
:10A950008DF87C008DF80310ADF810504FF4967010
:10A960002B492290059144F2506023902948299068
:10A97000264869462030FCF7CEFD08B1FCF714FAF2
:10A98000224801212030FCF7C3FD04F057F904F000
:10A990001BF81C216846FBF790FD4FF42030CDE9F1
:10A9A00000404FF47020029018488DF80C50643825
:10A9B0008089ADF80E0018480590184806908DF86B
:10A9C00010406846FDF752F808B1FCF7EDF902F0C7
:10A9D000A7FF1348008805EB004000E00FE011A13D
:10A9E00001F038FAFCF7BAFA3046FCF7FBF800BF82
:10A9F00001F020F90028FBD101F0D0FBF8E7012697
:10AA000078E700002185020051960200EC2E00201C
:10AA1000B02B002031CE02007DCE0200EB8B020075
:10AA2000F82D0020486561727420526174652053CE
:10AA3000656E736F72206578616D706C65207374DC
:10AA400061727465642E000070B5144682880E46EB
:10AA500005462088111D0144921C994201D8FE2A06
:10AA600001D90C2070BD521C32542088FF21401C9B
:10AA700080B2208031542088401C80B2208081190F
:10AA8000288804F00FFF2188084480B22080AA881B
:10AA900042B1A96841B13044FBF7E8FC2088A9889D
:10AAA00008442080002070BD072070BD2DE9F047CC
:10AAB000C7880446181D16468946B0FBF7F1B0FB5F
:10AAC000F7F207FB12009A193A44D21CB2FBF7F2D4
:10AAD000DDF820A001E02468491E0029FBD13D1AC1
:10AAE0008846B54216D818E0BAF1000F05D02118F3
:10AAF00009EB08002A46091D04E0204409EB08017F
:10AB00002A46001DFBF7B2FC00202468761BA844EF
:10AB1000B74201D9354600E03D46002EE4D1BDE8FC
:10AB2000F087000030B5024659B101F031FA00213A
:10AB3000074C09E004EB810315685B88AB4202D146
:10AB40001160002030BD491C8142F3D3052030BD87
:10AB5000C42D0020F8B50F4601781446054601299A
:10AB600001D1687830B12088821C9A422DD8012901
:10AB700002D006E00720F8BD69780144891C99429B
:10AB800023D8181A801E86B2ADF800602188B81C40
:10AB9000084469467DDF0028EDD12878022805D1D8
:10ABA000BDF80010B14201D809210AE008210128AE
:10ABB00005D16878B04202D8ADF8000001E0ADF8E8
:10ABC0000060BDF80000FE2801D90C20F8BD2288E5
:10ABD000401CB8542088401C80B220803954208802
:10ABE000401C2080BDF80010084420800020F8BDE3
:10ABF00070B505460C004FF0FF0020D04FF6FF76F1
:10AC0000B5421CD00E48012241782846FCF7D6FFF9
:10AC10002846FEF70BFFFF2803D1FEF723FFFF288E
:10AC20000DD0084B00EB400203EB82014D8023F86E
:10AC3000226022684A60A2880A81A2798A7270BD65
:10AC4000EE2B002028310020034A00219268C0E941
:10AC500000218160704700001C2C002070B54FF669
:10AC6000FF750E46A84201D1002000E0401C84B2CE
:10AC700008E02146304603F002F808B1204670BDD6
:10AC8000641CA4B2FF2CF4D9284670BD10B5FBF7A4
:10AC90000CFB08B1002010BD112010BD10B531B162
:10ACA000B2FBF3F403FB14241CB1092010BD0E20E9
:10ACB00010BD01600021416081608281C38108462E
:10ACC00010BD70B50C460546FBF7A4FA002802D06B
:10ACD00021882868084470BD10B50A8849888A42CE
:10ACE00003D1FBF7D9FA012010BD002010BD70B5CB
:10ACF0000C460546FBF7B3FA002802D061882868A5
:10AD0000084470BD10B50A8849888A4203D1FBF710
:10AD10009DFA012010BD002010BD01F01F0301228B
:10AD20009A40D243490900EB8100114600F059B81E
:10AD30000A4601F01F030121994010B552090C4643
:10AD400000EB820000F05DF8204000D0012010BD33
:10AD50002DE9F04180460D460024481E012101EBFB
:10AD6000501716E058F82400C04390FAA0F0B0FA4B
:10AD700080F020280CD200EB4416AE4208D23146B7
:10AD80004046FFF7D5FF0028ECD13046BDE8F08102
:10AD9000641CA742E6D82846F8E74A0950F8220082
:10ADA00001F01F0201219140084000D001207047AE
:10ADB00001F01F0301229A40490900EB810011466E
:10ADC00000F029B8002100F017B8012100F023B8E5
:10ADD000012100F016B808B56A46FBF7B2FA0098F0
:10ADE00008BD08B56A46FBF792FA009808BD08B599
:10ADF0006A46FBF7A6FA08BD08B56A46FBF787FA6C
:10AE000008BD08B56A46FBF775FA08BD08B56A467D
:10AE1000FBF764FA08BD08B56A46FBF76BFA0098C1
:10AE200008BD08B56A46FBF799FA009808BD38B521
:10AE3000044600258DF800506846FCF751F821685B
:10AE40006268086890420ED9401E08600178A38AA3
:10AE5000E26801FB0325227A2168101AC0B20A7940
:10AE6000824200D208719DF80000FCF75DF8284688
:10AE700038BD38B5054600208DF800000C46684600
:10AE8000FCF72EF8E868A98A201AB0FBF1F12A68CD
:10AE90001068431C136001709DF80000FCF744F833
:10AEA00038BD10B530B1017A42680368891AC9B259
:10AEB0001A6006E00E2010BD03681A68541C1C605E
:10AEC0001170491EC9B2F7D200680021017108460D
:10AED00010BDC20800F007030120895C98400840BB
:10AEE000704710B5C20800F00703885C01249C403D
:10AEF0002043885410BD10B560B10161F72120F8DE
:10AF0000021B20F8021BFB2100F8021BFFF7EEFAE0
:10AF1000002010BD0E2010BDF0B5858893B00C4602
:10AF2000002D39D1018800263E4F24293BD006DC74
:10AF3000102909D011290CD0232958D14FE03A29E2
:10AF40000BD0552953D129E00146204601F0A4FF3A
:10AF50004DE0A01DFFF7CAFA49E02246408934F8C7
:10AF6000061F814200D808466080172800D21720AB
:10AF70006080106970B1607960B1D7E90001CDE9F6
:10AF80000301ADF80E506088ADF81000136903A9F5
:10AF9000104698476671267113B0F0BD01462046F1
:10AFA00001F0CAFF23E0011D2C2206A8FBF75EFA80
:10AFB000BDF81800BDF81C2004EBC0014A732269DB
:10AFC000AAB1D7E90423CDE90423ADF81200487BE8
:10AFD0008DF814002269204604A9904707E0017A01
:10AFE000207B884200D201462846FDF747FEA07A22
:10AFF0000028D1D0E1882846A5DF012570B11128AD
:10B00000CAD001F065FB0246074808A1008813B0CA
:10B0100005EB0040BDE8F04000F020BFA672E572ED
:10B02000BAE7000028000300C42D002073645F62AB
:10B030006C655F67617474635F65786368616E6790
:10B04000655F6D74755F726571756573742829200D
:10B0500072657475726E65642025732E00000000A1
:10B0600020B10278DE2A03D0082070470E207047F6
:10B0700041800020704760B159B10278DE2A0AD0C1
:10B0800009684160DE2101704FF6FF7141800020A8
:10B0900070470E207047082070477FB5054600298D
:10B0A0004DD0002D4BD008780C46DE2847D1A8881B
:10B0B0006188884202D1204604F0B4FC2888012827
:10B0C00025D002283BD011283AD0512837D135F865
:10B0D000040F6188884232D1A978A81C02292ED198
:10B0E000017A042903D0062901D0052927D100219E
:10B0F000009102228DF8002001914FF4C07202915C
:10B100000391ADF80420007A05280FD010E0297AC9
:10B110002046012913D1A988428891420FD10121EB
:10B12000017204B0BDE8704004F07CBCADF80410BE
:10B1300028886946B0DF002801D0616888477FBD54
:10B14000A88861888842FAD14FF6FF7060807FBD81
:10B1500000F180400068002800D00120704708B549
:10B1600000F18040002101600068009008BD0000EF
:10B1700070B50B4C207808B185250FE00020A06049
:10B1800060602061E060074801F0DEFA054601F0EA
:10B1900029FA08B901F0C2FA01202070284670BDD2
:10B1A000843300205D8A020038B500258DF80050F8
:10B1B0006846FBF795FE074CE068401EE060E068DB
:10B1C00010B901F0D1FAA5709DF80000FBF7ACFEB4
:10B1D00038BD000084330020F0B5054604781548DA
:10B1E00089B0164640F82420124A0869121DA2F1BF
:10B1F000080742F82400487F385520226846FBF7AC
:10B2000035F904942878385C48B10EB10A4A00E058
:10B2100000226946281D01F027FD09B0F0BD0EB1DE
:10B22000064A00E00022694605F10C0001F0EEFB41
:10B23000F3E70000802C002081F70200CDF502002A
:10B240000FB408B50399002904D004AA00926A46F5
:10B2500000F00FF801B05DF814FB10B582680446E9
:10B26000002A05D0D4E90403216898470020A06093
:10B2700010BD2DE9FC4791460C00804676D014F8AD
:10B28000011B39B125290ED04046FDF70FFB207870
:10B290000028F4D198F80C00002867D04046BDE89B
:10B2A000FC47FFF7DABF0020012221782B291BD0B1
:10B2B0002D2902D0302908D102E040F0010001E040
:10B2C00040F00200641C002AEFD100252A290ED08C
:10B2D0002178A1F130020A2A11D205EB850201EB97
:10B2E0004205641C303DF1E740F00400EAE7D9F87C
:10B2F00000100B1DC9F800300968641C0D4421784A
:10B3000000232E290BD114F8011FA1F130020A2AC3
:10B3100005D203EB830201EB4203303BF3E76C29D8
:10B320000DD068290BD0692921D00BDC252918D034
:10B33000582931D063290ED0642915D117E014F8AB
:10B34000011FECE7702969D0732932D075291BD011
:10B35000782909D120E0D9F80000011DC9F80010B2
:10B3600001784046FDF7A2FA641C90E76CE0D9F83A
:10B3700000100A1DC9F800200968CDE900500A2212
:10B380004046FEF79DFFEFE7D9F800100A1DC9F807
:10B39000002009680A2206E0D9F800100A1DC9F841
:10B3A000002009681022CDE90050404604F090FAD0
:10B3B000DAE7D9F8001000270A1DC9F800200E6846
:10B3C000C00705D112E04046761C7F1CFDF76EFADF
:10B3D00031780029F7D104E0202140466D1EFDF7A9
:10B3E00065FABD42C0D9002DF6D1BDE74EB1304659
:10B3F000FBF76EF8074604E0202140466D1EFDF77E
:10B4000055FABD4206D9002DF6D103E04046761C20
:10B41000FDF74CFA31780029F8D1A5E7D9F80000FA
:10B42000011DC9F80010056830214046FDF73EFABD
:10B4300078214046FDF73AFA08200021CDE90001C5
:10B44000034610222946B0E7BDE8FC872DE9F84FF6
:10B450002B4E04009A4630884FF00103154689466A
:10B4600003EB004024D0216800292BD0002D32D0DE
:10B47000626849464FF010071268A2F1010C1CEAFD
:10B48000090F11D198466A432046FBF783FB002839
:10B490002AD0206853462A46066901B0494620460C
:10B4A000B446BDE8F04F6047164B17A2009721E065
:10B4B0000E210091134B1EA21FA100F0DEFC0E20F6
:10B4C000BDE8F88F082100910E4B26A21AA100F0CA
:10B4D000D4FC0820F4E7092100910A4B24A216A10C
:10B4E00000F0CBFC0920EBE700973188054B214A9F
:10B4F00008EB014010A100F0C0FC1020E0E70000C4
:10B50000E82D00206B010300616464725F69735F62
:10B51000706167655F616C69676E656428705F66FE
:10B52000732C20706167655F61646472290000009C
:10B53000705F667300000000257320636865636BAD
:10B54000206661696C656420696E20257328292056
:10B55000776974682076616C756520307825782E5F
:10B5600000000000705F66732D3E705F61706900BF
:10B570006C656E000C05030038B503000F484FF0F2
:10B5800001054FF00E04008805EB004009D061B1C1
:10B5900019600C6801B0A446BDE830401146184659
:10B5A0006047074B07A2009402E0054B07A20094F6
:10B5B00008A100F062FC0E2038BD0000E82D00203C
:10B5C00020010300705F667300000000705F61700F
:10B5D00069000000257320636865636B20666169FC
:10B5E0006C656420696E202573282920776974684A
:10B5F0002076616C756520307825782E000000007B
:10B600002DE9F04128B1016819B1C969BDE8F041DF
:10B6100008470D4D0D480024461B14270DE000BFC0
:10B6200004EB840005EB8000016829B1C9698847F3
:10B6300010B10120BDE8F081641CB6FBF7F0A04218
:10B64000EED80020F6E70000B02D0020C42D002029
:10B65000044801214174007A08B10020704701209C
:10B6600070470000E8360020012801D0032808D1E7
:10B670000449002201284A7400D00020087402F016
:10B6800073BD7047E836002070B50246022801D02D
:10B69000032A45D1234C207A002841D0012833D0F9
:10B6A000022831D120480023022A006802D0032A50
:10B6B0002AD11BE0E360017911B1012924D10DE009
:10B6C000D0E90565711B4FF48056B14200D3314675
:10B6D000294481614569A9420ED015E00169491CE0
:10B6E0000161426991420FD1237213E0E168491C64
:10B6F000E160082908D9E3602372022A0AD00D21EB
:10B70000FDF786FC02F0D6FC607C28B1BDE87040F5
:10B7100000F06EBF0021F3E7BDE8704002F024BDE9
:10B7200070BD0000E8360020242D00202DE9F84FE0
:10B730003A4D04008B4628884FF00106DDF828A01A
:10B74000984691464FF00E0106EB00401AD0B9F131
:10B75000000F1BD02168002920D00921B8F1000F6B
:10B7600025D062685368B8FBF3F703FB1782002A01
:10B7700021D02B4B2BA2009135A100F07EFB09209C
:10B78000BDE8F88F264B3DA2009102E0244B3DA27C
:10B7900000912FA100F071FB0E20F1E7082100912C
:10B7A0001F4B3AA22AA100F068FB0820E8E71C4BD7
:10B7B00039A20091E0E75846FBF7E6F9102798B167
:10B7C0004846FBF7E1F9B0B1424659462046FBF73F
:10B7D000E1F9B8B1CDF800A0206843464A46C568F3
:10B7E00059462046A847CBE7009728880C4B06EB24
:10B7F00000402AA20CE000972888094B06EB004085
:10B800002CA205E000972888054B06EB004032A2E9
:10B810000FA100F032FB1020B2E70000E82D00205D
:10B820005801030021286C656E202520705F667327
:10B830002D3E705F666C6173685F696E666F2D3E4A
:10B8400070726F6772616D5F756E697429000000B8
:10B85000257320636865636B206661696C6564208D
:10B86000696E202573282920776974682076616CB9
:10B87000756520307825782E00000000705F6673B3
:10B8800000000000705F737263000000705F6673F9
:10B890002D3E705F617069006C656E00616464725A
:10B8A0005F69735F616C69676E65643332286465D4
:10B8B00073742900616464725F69735F616C6967A6
:10B8C0006E65643332282875696E7433325F74296B
:10B8D000705F737263290000616464725F69735FF3
:10B8E00077697468696E5F626F756E647328705FE4
:10B8F00066732C20646573742C206C656E290000BF
:10B9000070B541EA4201DDE904564FF0A04441EA36
:10B91000830141EA052104EB800041EA0641C0F8B9
:10B92000001770BD70B541EA4201DDE904564FF0E1
:10B93000A04441EA830141EA052104EB800041EA89
:10B940000641C0F8001770BD70B541EA4201DDE95B
:10B9500004564FF0A04441EA830141EA052104EB7B
:10B96000800041EA0641C0F8001770BD70B541EA99
:10B970004201DDE904564FF0A04441EA830141EA67
:10B98000052104EB800041EA0641C0F8001770BDB4
:10B990001CB5002100910B4601220191FFF7D4FF55
:10B9A0001CBD1CB5002100910B4601220191FFF73F
:10B9B000DDFF1CBD1CB500220B4600921146019212
:10B9C000FFF7C2FF1CBD1CB500220B4600921146BA
:10B9D0000192FFF7CBFF1CBD1CB5002100910B4667
:10B9E000012201911146FFF7AFFF1CBD1CB50021DC
:10B9F00000910B46012201911146FFF7B7FF1CBDD4
:10BA00004FF0A04202EB8000D0F8002722F4403231
:10BA1000C0F80027D0F8002742EA0141C0F800171B
:10BA2000704701224FF0A043824011B1C3F80825AE
:10BA30007047C3F80C25704718B5084B6C46014495
:10BA40001B68009306E000BF54F82030D3F810358F
:10BA5000401C08C28142F7D818BD0000D000030086
:10BA6000034908B50844002101600068009008BD42
:10BA70000060004002494058012800D00020704773
:10BA80000060004030B5124B01460020D3F810444E
:10BA9000224609E0157A854205D1401C0A28F7DBC9
:10BAA0004FF0FF3030BD5268002AF3D1421CF9D06C
:10BAB0000872D3F810242AB152684A60D3F81024CF
:10BAC000516030BD0022C3F810144A6030BD000040
:10BAD00008380020F0B595B01C4615460F460846BC
:10BAE0001A9E00F025FB182109A8FAF7E6FC0E962D
:10BAF000CDE909540023082203A9384600F02DFBA4
:10BB000005980690BDF81000ADF81C00BDF81200B5
:10BB1000ADF81E0000208DF821000398082600F0E3
:10BB20000300012802D0022818D032E003983346DF
:10BB3000850AC0F3C2008DF8200003980FA9C0F356
:10BB40008314A200384600F008FB09A8009006AB59
:10BB500022460FA9284600F047FA1AE00398840D00
:10BB6000C0F3C2008DF82000082C01D2254600E069
:10BB7000082533462A460FA9384600F0EEFA2E442F
:10BB8000641B09AB06AA29460FA800F07FF9002C18
:10BB9000EAD1384600F0D2FA15B0F0BD7047012066
:10BBA00003F032BD084810B50178084A515C19B15C
:10BBB000001D01F0E5F802E00C3000F0F3FFBDE8F5
:10BBC0001040002003F020BD382D00207C2C0020E8
:10BBD00008B5034A00924023024AFFF77BFF08BDE5
:10BBE00091EA0200083700200A4A012902EBC0004E
:10BBF00007D0022907D0032907D0042907D0002045
:10BC000070470220704704207047007970474079E0
:10BC100070470000580C030010B5FFF7C0FF042167
:10BC20000348FFF72FFF02490120487210BD0000B2
:10BC30004C2D00202DE9F04F8DB0FCF747FE18B1D8
:10BC400000200DB0BDE8F08F7A4C4FF0000BC4F827
:10BC500018B4BFF34F8F60680290A568D84628409B
:10BC600004EB800008E021680298814201D86160FD
:10BC7000E6E7284004EB80000C3002A9FEF7B4FB95
:10BC80000028F0D105AA029901EA050304EB830319
:10BC9000491CDB6842F82030401C02910228F2D394
:10BCA000059800F00300022802D001284ED0A9E038
:10BCB00005985022810D8946B2EB905F00D8502143
:10BCC0000E4666F39F50059008315B4800F0E7F997
:10BCD000070079D000F02CFA4346082205A938461F
:10BCE00000F041FA029908F1080A2940681A800018
:10BCF000001D864223D94F4D0C3530B1C2B204EB42
:10BD00008101301A90460C3104E02946F2B2002538
:10BD100090462846C6B25346384600F024FA0AEB4D
:10BD200008032DB1324629464FEA070000F01BFAFE
:10BD3000029909F1030001EB900002903BE004EB53
:10BD400081015346324638460C31EFE70598C0F37F
:10BD50008310062800D30620059960F38911C1F3EA
:10BD60008310801C05918100334800F098F907008A
:10BD700048D000F0DDF94346082205A9384600F016
:10BD8000F2F908F1080800260FE00298434600EA9D
:10BD90000501401C04EB81010290042238460C315D
:10BDA00000F0E1F908F10408761C0598C0F383104F
:10BDB000B042EAD847B1D4F81054D4F8180468B1A6
:10BDC000384600F0BBF92FE01CE0687A012804D166
:10BDD0002A6828463946126890476D68002DF4D1CC
:10BDE000384600F0ABF98DF800B06846FBF778F8FC
:10BDF000D4F8180408B9029860609DF80000FBF7B9
:10BE000093F811E0D4F8104404E0216820468968D2
:10BE100088476468002CF8D108480221008801EBAB
:10BE2000004007A100F016F8FCF750FD80F001007B
:10BE300007E7000008380020E00C0300F82D002080
:10BE40004261636B656E647320666C7573686564CC
:10BE50000000000000231A4603F00EBA08B50123C3
:10BE600000926A4603F008FA08BD1CB5CDE900232C
:10BE700002236A4603F000FA1CBD3EB5069C8DE81D
:10BE80001C0003236A4603F0F7F93EBD2DE9F04795
:10BE90000E4680461C46924608293ED894F80C90DF
:10BEA000002020731946104602F096F80025B5428E
:10BEB00006D218F805201AA12046FFF7C1F903E0C1
:10BEC00019A12046FFF7BCF96D1C082DEFD317A16F
:10BED0002046FFF7B5F90025B54210D218F80570D5
:10BEE000FAF7C0FA0068C05D10F03E0F01D03A4684
:10BEF00000E02E220EA12046FFF7A2F903E00DA1DB
:10BF00002046FFF79DF96D1C082DE5D3012221463F
:10BF1000504602F043F884F80C90BDE8F08700002A
:10BF20002025303278000000202020007C00000016
:10BF30002563000020000000104810B5FF2181603B
:10BF4000002101604160C0F81814C0F8141480F892
:10BF500020140B4800F0F0F800280DD109480A49D8
:10BF60000A4B401AC108002003E000BF23F820005C
:10BF7000401C8842FAD3002010BD00000838002081
:10BF8000E00C0300E00C0300580C0300C42D00205B
:10BF900002480349401AC00870470000E00C030043
:10BFA000580C030013B56846FEF7BCFD08B100202D
:10BFB0001CBD0248009950F831001CBD580C03000C
:10BFC00070B508480125D0F8104480F8205405E0E9
:10BFD000657221682046496888476468002CF7D15B
:10BFE00070BD0000083800202DE9FF4781460C9DF8
:10BFF00000200C462F7B2873984616462946184683
:10C0000001F0EAFF072E42D2DFE806F004090F161E
:10C010001F2A360049462846FFF712F937E04946FD
:10C0200028462268FFF70CF931E0D4E9002349469D
:10C030002846FFF705F92AE0A0680090D4E900231C
:10C0400049462846FFF7FCF821E0D4E90201CDE992
:10C050000001D4E9002349462846FFF7F1F816E02D
:10C0600004F1080007C88DE80700D4E90023494619
:10C070002846FFF7E5F80AE004F108000FC88DE84C
:10C080000F00D4E9002349462846FFF7D9F80022DB
:10C090002946404601F082FF2F73BDE8FF872DE956
:10C0A000F041858A80462D1F4819C01CB0FBF5F071
:10C0B000C6B24046FEF7BBFE041E19D00020207118
:10C0C00001206071E58000272546761EC4F80080B7
:10C0D0000BE04046FEF7ABFE60B16179491C61712F
:10C0E000286005467F1CC0F80080B742F1D3204687
:10C0F000BDE8F081204600F002F80020F8E72DE9C5
:10C10000F041457901466B1E002201E00968521C8E
:10C110009A42FBD30F680146002605E038460C68BA
:10C12000FEF7A7FE2146761CAE42F7D3BDE8F081AC
:10C130000121001DFEF74FBEFEF7B3BE10B5044649
:10C140000121001DFEF76DFE10F0FF0F04D1204607
:10C15000BDE81040FFF7D3BF10BD38B501240094EF
:10C16000FEF7A4FC38BD38B500240094FEF79EFC11
:10C1700038BD0000064910B500204870091D086050
:10C18000BFF35F8F0349044800F05EFA002010BD42
:10C190002C2D0020C8010300FC36002008B500202B
:10C1A0008DF800006846FAF79BFEF1EE100A20F0C9
:10C1B0009F00E1EE100ABFF35F8F08494020C1F8ED
:10C1C00080029DF80000FAF7AFFE00F00BFA08B10C
:10C1D00041DF08BD20BF40BF20BF08BD04E000E034
:10C1E000FAF7E2BD20B103490968016000207047F9
:10C1F0000E207047B40303002DE9FE4306460D46AA
:10C200000846FFF7EFFF00287ED18046CDF800807A
:10C21000CDF8048001244FF4A0708DF80060ADF8D3
:10C220000400CDF808808DF80240694620202A6875
:10C2300069DF404F40B100F04BFA024638883E4972
:10C2400004EB0040FFF70AFECDF800808DF80140B6
:10C250008DF80280CDF80480CDF808808DF8038039
:10C26000694640202A6869DF40B100F031FA024691
:10C270003888324904EB0040FFF7F0FDCDF800802C
:10C280008DF80060F720ADF80200CDF80480CDF8FD
:10C290000880694623202A6869DF40B100F018FA57
:10C2A00002463888264904EB0040FFF7D7FDCDF859
:10C2B0000080CDF80480CDF808808DF800804646D7
:10C2C000694601202A6869DF40B100F001FA0246A0
:10C2D00038881C4904EB0040FFF7C0FD4FF4B06004
:10C2E0000090019602966946A1202A6869DF40B154
:10C2F00000F0EEF902463888134904EB0040FFF7DE
:10C30000ADFD0096019600E011E002968DF8004028
:10C310006946A0202A6869DF40B100F0D9F90246D9
:10C3200038880A4904EB0040FFF798FD0020BDE87B
:10C33000FE830000002E0020A40A0300EC0A030084
:10C34000380B0300040A0300500A0300B00903007D
:10C350002DE9F0410446D0F8008060DF2168194DD6
:10C36000074641451CD92888022606EB004016A145
:10C37000FFF770FD2888424606EB00401EA12368A7
:10C38000FFF773FDF006D0F80C012168800200F180
:10C390000050421A288825A106EB0040FFF75EFDF9
:10C3A000012467B1384600F093F9024628882AA193
:10C3B00004EB0040FFF752FD3846BDE8F0812E48FF
:10C3C0000470F9E7002E0020496E73756666696394
:10C3D00069656E742052414D20616C6C6F636174AD
:10C3E000656420666F722074686520536F667444BC
:10C3F00065766963652E00004368616E6765207429
:10C4000068652052414D207374617274206C6F63B3
:10C410006174696F6E2066726F6D203078257820A8
:10C42000746F20307825782E000000004D61786907
:10C430006D756D2052414D2073697A6520666F726B
:10C44000206170706C69636174696F6E206973201C
:10C45000307825782E00000073645F626C655F653C
:10C460006E61626C6528292072657475726E6564F0
:10C470002025732E00000000AB2D002030B515489C
:10C48000ADF5017D0078002821D04FF4FA7500BF8A
:10C49000ADF8005280A9684661DF38B1052816D092
:10C4A0000DF5017DBDE83040FAF77EBC6C460A49C7
:10C4B0007DA800F0C9F806E0D0E9002120469047A9
:10C4C0007DA800F0D8F87F980028E1D0F4E70DF5BA
:10C4D000017D30BDAB2D0020B8030300F8B5134C2F
:10C4E0002078C0B10120A07002F0DEF8112814D02D
:10C4F000022002F0F1F800258DF800506846FAF7A6
:10C50000EFFC11DF064625709DF80000FAF70CFDE0
:10C510002EB13046F8BD0820F8BD0020F8BDA5704A
:10C5200002F066FE032002F0D7F8F6E7A82D0020FF
:10C530007CB5204C207808B108207CBD0120A0707B
:10C54000002002F0B1F8112819D0002002F0C4F840
:10C5500019480026006801908DF800606846FAF7D7
:10C56000BFFC164901A810DF05000AD0002020708A
:10C570009DF80000FAF7D8FC2DB128467CBD0020BC
:10C580007CBD0120F3E7A67066700721162002F03B
:10C5900041F808B1FAF708FC0721152002F03AF833
:10C5A00008B1FAF701FC02F03FFE012002F094F816
:10C5B000E5E70000A82D00204C0303002D6D0200CC
:10C5C0000EB50749684600F03FF805E0D0E90010D5
:10C5D0008847684600F04FF802980028F6D10EBD53
:10C5E000680303000148007870470000A82D002070
:10C5F0000548817819B1007818B1FFF76FBF08209E
:10C600007047FFF795BF0000A82D00201FB56846B2
:10C610004BDF30B1052814D004B0BDE81040FAF764
:10C62000C3BB084901A800F00FF806E0D0E90021DB
:10C630000098904701A800F01EF803980028E6D063
:10C64000F4E71FBDD4030300016009684160AFF344
:10C65000008010B5D0E900215368994201D1002132
:10C6600004E0D1E90034A34202D01946816010BD34
:10C6700008314160F0E7816800290BD002689268B8
:10C680000A44826041684B689A4203D10831416094
:10C69000FFF7DFBF704700000C4A10B502F5947336
:10C6A0000EE0991AC91001EBD171491002EBC101DA
:10C6B0000C68844201D90B4602E005D201F1080260
:10C6C0009A42EED3002010BD486810BDE801030077
:10C6D00000B5FFF7E1FF002800D1014800BD0000D0
:10C6E000D40103004058002800D00120704708B54D
:10C6F000002242504058009008BDD0F80403084082
:10C7000000D0012070474058002800D00120704719
:10C7100008B5002242504058009008BD0848006803
:10C72000012110F0010F08D14FF0E020E02280F845
:10C730000024C0F88012C0F8001102480160704760
:10C7400000E100E0180500400649024600200B7990
:10C750000BB1852070470A6001220A7100224A71DC
:10C7600070470000882C002004490120086004481C
:10C770000168C1F300410029FAD170470C00004064
:10C7800018040040002802D0014980010847704782
:10C79000F10003002DE9F0418846054601F008F953
:10C7A000234E002828461AD0FCF7D0F8304490F8E1
:10C7B00048008009032802D001280ED007E04FF07E
:10C7C000A040D0F81005E84010F0010F05D003217B
:10C7D0002846BDE8F041FFF713B90221F8E701F060
:10C7E000F3F8002822D02846FCF7B0F804464FF4AE
:10C7F000807000EB84000F4F81B207EB8400D0F80B
:10C80000102542F00102C0F810250846FFF728F96C
:10C81000B8F1000F0AD02846FCF798F856F8200027
:10C82000002803D00120A040C7F80403BDE8F08130
:10C8300098330020006000402DE9FC41DFF8BC8007
:10C84000044608EB0400002790F930001346C01797
:10C850000E46401C01D008274CE0B0781946C0F3C2
:10C8600040022046FCF74EF80546401C41D0B07807
:10C87000410719D4C0070AD04FF0A04000EB840153
:10C88000D1F8000720F00200C1F8000707E00021FE
:10C890007378204600910A460191FFF743F8174943
:10C8A00020465431FEF71DFBB078800718D5144898
:10C8B000317800EB8500D0F81025124B1A40C0F8F3
:10C8C00010254FF4F8524FF4403302EA042203EAF1
:10C8D00001410A43D0F810150A43C0F8102509E0B9
:10C8E00008EB0500327810F8481F41EA8211017008
:10C8F00000E004273846BDE8FC81000098330020A2
:10C9000000600040FFE0FCFF4FF0A041D1F810159F
:10C91000C14011F0010000D00120704770B5184DE2
:10C9200095F8580008B1082070BD0020411E2A1853
:10C93000401CC0B282F830102028F8D300242046D2
:10C94000FBF7D2FF641CE4B20C2CF8D300240D4991
:10C95000E0206C6581F8000401264020891FC1F8A1
:10C960008002C1F800014FF4BE70FFF779F8064964
:10C97000F007C1F8040385F85860204670BD000038
:10C980009833002006E000E000600040034890F883
:10C990005800002800D00120704700009833002084
:10C9A0000121B1EB507F01D1012070470020704779
:10C9B00038B50D4601F05CFB040014D000208DF862
:10C9C00000006846FAF78CFA207928B19DF800003B
:10C9D000FAF7AAFA112038BD0120256020719DF8D0
:10C9E0000000FAF7A1FA002038BD10B501F040FBB5
:10C9F000002802D000210160017110BD01490248E8
:10CA000002F02ABEF4330020002000402DE9F0415E
:10CA10000546007916460F4600EB40012D4A01EB12
:10CA2000C00102EB810494F82A1011B10820BDE87E
:10CA3000F081294951F820102868FFF7B9FF08B1A3
:10CA40001120F4E739462846FAF7B4FA66603869E7
:10CA5000206030004FF001062FD03F7F4FF48E71E1
:10CA60002868FFF744FE4FF4A2712868FFF73FFEE5
:10CA700028681A49C0F8041328684FEA4711000BC8
:10CA800040B2002806DA00F00F0000F1E02080F844
:10CA9000141D03E000F1E02080F800142868000B6A
:10CAA00040B200F01F0206FA02F14009800000F1D6
:10CAB000E020C0F88012C0F8001128680421C0F8F6
:10CAC00000150020A061E06184F8290044F8140FEB
:10CAD000A675ACE7F4330020D40003008000020008
:10CAE0002DE9F047054600790B4600EB400101EBCC
:10CAF000C000234901EB8004284600F043F810B140
:10CB00001120BDE8F0874FF00008C4F82080A36032
:10CB1000626184F828804FF48E7647463146286853
:10CB2000FFF7E5FD28684FF00109C0F8089021469D
:10CB3000286802F02DFD606800BBD5F800A00EE06B
:10CB400094F8280008B10F2716E031465046FFF749
:10CB5000C9FD0028F4D02146504602F019FD216A93
:10CB600060698142F1D331462868FFF7BBFD002898
:10CB7000F9D02868C0F80C90C4F814803846C0E793
:10CB8000F4330020007900EB400101EBC0000449C0
:10CB900001EB80004069002800D0012070470000B0
:10CBA000F43300202DE9F047044600794FF00009E6
:10CBB00000EB400101EBC000254901EB8007206834
:10CBC000C0F80095786880B120682249C0F8081341
:10CBD00020680121000B40B200F01F029140400983
:10CBE000800000F1E020C0F880112068D0F80C250A
:10CBF000D0F81485D0F80865D0F810554FF0FF3103
:10CC0000C0F81415C0F80C152068C0F80815C0F855
:10CC10001015501C02D01046FEF7BAFEB8F1FF3FC7
:10CC200002D04046FEF7B4FE681C02D02846FEF74C
:10CC3000AFFE701C02D03046FEF7AAFE2068FFF758
:10CC4000D4FE87F82A90C7F80490BDE8F08700006A
:10CC5000F4330020840202000149024802F0A8BD1A
:10CC600020340020002000402DE9F0410546164602
:10CC700000790F46154A00EBC00102EB810494F8DD
:10CC8000201011B10820BDE8F081114951F82010A1
:10CC90002868FFF78DFE08B11120F4E739462846D1
:10CCA000FAF7CCF96660386920601EB1397F2846F2
:10CCB000FDF75AFB28680821C0F800150020A06184
:10CCC000E0610121606184F82010DCE7203400205D
:10CCD000D80003002DE9F04704460E4600792049AC
:10CCE00000EBC00001EB800517463046FFF758FE09
:10CCF00030B1204600F036F820B11120BDE8F087B1
:10CD00001020FBE76F61AE604FF49076002731464C
:10CD10002068FFF7FDFC4FF4AC7841462068FFF730
:10CD2000F7FC2068AA686969C0F84425C0F848156E
:10CD3000206801218160686878B9B1464946206859
:10CD4000FFF7E1FC064641462068FFF7DCFC06439E
:10CD5000F4D000B10F27002068613846CEE700000C
:10CD6000203400200079054900EBC00001EB800071
:10CD70004069002800D001207047000020340020C6
:10CD80002DE9F04704460079274900EBC00001EB8C
:10CD9000800720684FF00009C0F80095786880B1DE
:10CDA00020682249C0F8081320680121000B40B216
:10CDB00000F01F0291404009800000F1E020C0F81F
:10CDC00080112068D0F80C25D0F81485D0F80865BB
:10CDD000D0F810554FF0FF31C0F80C15C0F81415FD
:10CDE0002068C0F80815C0F81015501C02D0104675
:10CDF000FEF7D7FDB8F1FF3F02D04046FEF7D1FD68
:10CE0000681C02D02846FEF7CCFD701C02D03046CC
:10CE1000FEF7C7FD2068FFF7E8FD87F82090C7F808
:10CE20000490BDE8F08700002034002010030200C9
:10CE300010B590B1032814D10A480321008801EBF2
:10CE4000004009A1FFF706F80220FBF7B1FB00281C
:10CE500007D0BDE81040F9F7A7BFBDE8104001F0CA
:10CE60009BBF10BDF82D002046617374206164766D
:10CE70006572746973696E672E000000007800287F
:10CE800007D104483B21408876DF002801D0F9F71C
:10CE90008BBF7047902B002070B58D88027900EB16
:10CEA000C5042273C97BA41D012902D0022904D123
:10CEB00001E0008800E0408820802188608881426D
:10CEC0000FD92846A5DF0126A0B1112814D0FFF7FD
:10CED000FFFB02460A480BA1008806EB0040FEF764
:10CEE000BDFFA179E079814208D92846BDE87040AC
:10CEF000FBF7C4BE6671F4E72671F2E770BD00006F
:10CF0000C42D002073645F626C655F676174746335
:10CF10005F65786368616E67655F6D74755F726584
:10CF2000717565737428292072657475726E6564F5
:10CF30002025732E000000007CB506468D88C88829
:10CF400006EBC504A41D172800D2172021888142B2
:10CF500000D8084660800020207121882846B5DF6F
:10CF600050B1FFF7B5FB02460E480121008801EBE6
:10CF700000400DA1FEF772FF6079002810D13069E2
:10CF800000280DD01449D1E90201CDE90001ADF826
:10CF900002506088ADF80400326969463046904717
:10CFA0007CBD0000C42D002073645F626C655F6708
:10CFB000617474735F65786368616E67655F6D74D3
:10CFC000755F7265706C7928292072657475726E50
:10CFD00065642025732E00002800030048B1064A2E
:10CFE0000168914205D140680449401802D00128E7
:10CFF00000D0032070470000DEC0ADDE02FEE10E6F
:10D000008A7D022A04D90289CB881A44D21C028163
:10D010004289C988511AC91E418170472DE9F041E2
:10D020000D460221904600F58056298000F1080443
:10D03000144F1BE031462046FCF734FE40B1B8F1F6
:10D04000000F02D0012288F80020022816D004E048
:10D05000A0687969884200D9786128886188084485
:10D06000C01C2880608804EB80040C3431462046C4
:10D07000FCF72BFE0028DDD1BDE8F0814FF4806085
:10D080002880F9E7E02C002008B500210091014636
:10D090000823024A0248FEF749FB08BD08010300C5
:10D0A000B02D002008B50020009004480823044A51
:10D0B00001680448FEF73AFB08BD0000082D002077
:10D0C00000010300B02D00202DE9F05F0025DFF8FE
:10D0D0000891DFF808B12C464FF00308AA462F4606
:10D0E000D9F80C0000EB07363046FFF777FF78B32E
:10D0F000012847D0032862D100204FF4806200BF8E
:10D1000056F82010491C0ED004EB84010BEB810271
:10D11000A8F10100566003221FFA80F80BF82120C5
:10D12000641CA4B24BE0401C9042E9D32C48016837
:10D1300079B104EB840102200BF821000BEB810193
:10D140004E600881254828304480641CA4B205E064
:10D1500007E00221066081804FF0010A45F00105D9
:10D160002DE004EB840100220BF821200BEB810160
:10D1700001F110024E6030460831FFF74FFF45F0D5
:10D180000205CDE7BAF1000F0CD0022004EB8401B8
:10D19000134A0BF821000BEB810112684A60641CF2
:10D1A0000881A4B20E480022011D06603046FFF738
:10D1B00035FF0B48808802280CD0082005437F1CCF
:10D1C000BFB2032F8CD3B8F1020F00D20025E8B212
:10D1D000BDE8F09F0420F1E7B02D002024360020A8
:10D1E000082D002001494978FAF7D0BC142C002002
:10D1F000002101F0D1BF30B585B00C4605218DF876
:10D2000000101546ADF80200FCF7A4FFADF80400CD
:10D210006846CDE90245FBF791FF05B030BD00003F
:10D2200070B5054D06460024304655F82410884751
:10D23000641C042CF8D370BD580003003EB5104D9B
:10D24000002400BF05EB041002F046FD641C022C14
:10D25000F8D30124502002210094CDE9011008499F
:10D26000084BB039A02201F1A00000F0E7FB08B1A3
:10D2700003203EBD0348401E847000203EBD0000D8
:10D28000D8320020012C002000F06CB900F06CB9FD
:10D2900070B504460025C168184A284602EB001301
:10D2A0009B688B4202D102EB001003E0401C022875
:10D2B000F4DB00202178082904D0092908D013299B
:10D2C00014D112E0617A89B980B102F015FD0DE048
:10D2D000617A59B950B100218160817B41F002012E
:10D2E000817307490120087003E001252046FFF7FC
:10D2F00097FF2846BDE8704000F0C2BFD83200203A
:10D30000002C002000F0E5B908B513889B000093BD
:10D310006B4600F05FF908BD002300F05BB938B53B
:10D3200005460024204609E08178284600F080F870
:10D3300010B1052800D003240098401C00906946D5
:10D34000284602F0B5FC0028EED134B9284600F09A
:10D35000C4F910B1072802D00324204638BD0724A1
:10D36000FBE71346002200F069B900002DE9F04701
:10D370001F0015460E46814604D0072E05D0082E04
:10D3800016D102E00E20BDE8F0878DB1022D0FD836
:10D3900000F0AEF960B14FF000083146484602F0A7
:10D3A0006DFC041E06D0207BA8420DD00F20EAE7BA
:10D3B0000720E8E7FF214FF6FF7002F05FFC041E34
:10D3C00006D0A0F80090A670607BFF2802D00CE089
:10D3D0001120D8E72946154800F002FB01462046F7
:10D3E0006173FF2913D04FF001082573617B0F484B
:10D3F00000F044FB02000DD0ABB23146384600F0DD
:10D4000007FAB8F1000F0ED0082E05D00BE002F09D
:10D4100063FCDDE70320B6E738886FF0050101EB18
:10D420008000796888800020ADE70000C8320020C5
:10D4300070B5002402F022FC05000BD0686820B112
:10D4400000F06FF9040000D00324284602F054FCD9
:10D45000204670BD052070BD70B515460C460729E5
:10D4600003D0082C01D0072070BD02F007FC28B1C2
:10D4700005808470BDE8704002F0BEBB052070BD21
:10D480007CB50D46072903D0082D01D007207CBDAF
:10D49000002602F0F3FB040002D0606810B11CE02B
:10D4A00005207CBD617B0F4800F0E8FA02004FF0D8
:10D4B0000000009001908DF8025010D0237B294687
:10D4C000684600F03DF9684602F084FB211D68467D
:10D4D00000F010F90646092801D030467CBD032033
:10D4E0007CBD0000C83200204FF6FF714180014929
:10D4F000096808474000030030B587B01748FBF7BC
:10D50000A9FF10B1032007B030BDFBF7C5FE08B17D
:10D510008620F8E700F0CEF9002002904CF20704D4
:10D5200003900EE0694604A8FBF75EFF0098808830
:10D53000A0F5404085B204A8FBF716FF284600F08E
:10D5400075F902AA04A92046FBF735FF0028E9D0A7
:10D550000349012008700020D5E700004D9102002A
:10D56000F42B002000F088B900F08CB970B586B0BB
:10D5700014460E46054600F03BF940B105F5404023
:10D5800080B20F4A6946FBF716FF40B902E001205E
:10D5900006B070BD03A96846FBF726FF08B100205E
:10D5A000F6E7A5700398408820800498606003988F
:10D5B0008088A0F5404030806846FBF7D5FEE6E75E
:10D5C000F82B002002480021416081607047000074
:10D5D000F42B0020F0B587B01D46144607460E46D2
:10D5E000FF280AD8084600F003F930B103AA3146F3
:10D5F000384600F0E5F840B902E0072007B0F0BD7A
:10D6000001A903A8FBF7F0FE08B10520F6E7A67014
:10D6100001984088208045B18200286890420BD351
:10D6200002996068F8F722FF01E00298606003A8A1
:10D63000FBF79AFE0020E1E70420DFE77FB586B024
:10D640001E460D460446FF282AD8A87800F0D0F8D8
:10D6500030B304F54040ADF80000A87803AA00F507
:10D660004040ADF802006868019028880290A978CF
:10D67000204600F0A5F80528089813D010B108A896
:10D68000FBF716FF694603A8FBF7D2FEB0B10728E7
:10D690001DD0082819D00E2817D003200AB070BD5D
:10D6A0000720FBE728B108AA694603A8FBF7CBFED1
:10D6B000ECE7694603A8FBF7C2FEE7E71EB1314677
:10D6C00003A8FBF788FE0020E8E71120E6E78620A4
:10D6D000E4E74FF6FF7000F0A9B810B5FF2801D9B4
:10D6E000072010BD00F0A8F800F02EF8002010BDB3
:10D6F00000F0F4B870B504460D46807800F078F874
:10D7000058B121882846FBF7BBFE002804D0072823
:10D7100005D0092800D0032070BD072070BD8620E9
:10D7200070BD01B56846FBF7C3FE002800D003209A
:10D7300008BD00000149C978FAF728BA142C002066
:10D740009BB200F065B8000070B51B4D8AB0002098
:10D75000687000904FF6FF760190304603E0204657
:10D7600000F07CF8204600F087F80446B0421DD057
:10D7700004F5404080B26A4602A9FBF724FE0A285D
:10D78000EDD004F5404080B2FBF746FD08280FD0ED
:10D7900000280BD005461422084905A8F8F766FEB4
:10D7A000ADF8184005A80795FFF79EFE0AB070BDBA
:10D7B00001206870FAE70000F42B00204400030009
:10D7C0007CB5054616460C46084600F011F80020C8
:10D7D000009005F54045019004F54044A8B2A1B27F
:10D7E0006B463246FBF7E0FD002800D005207CBDEB
:10D7F00007280BD0012809D0082807D0052805D014
:10D80000062803D0042801D000207047012070476B
:10D8100010B503EB83034FF6FF7404EA0313817022
:10D82000DB1C99084260018010BD00000149FBF734
:10D83000E5B80000F832002010B50446A0F57F409E
:10D84000FF3807D004492046FBF7D8F8A04201D1A1
:10D85000012010BD002010BD1833002010B5044673
:10D86000044900F029FE03492046BDE8104020315C
:10D8700000F022BEF83200200149FDF7EFB90000A8
:10D880001833002070B50A49FDF7E8F904464FF651
:10D89000FF7507E000F02CF838B105492046FDF788
:10D8A000DDF90446AC42F5D170BD204670BD0000E4
:10D8B000F832002010B508484021F8F7FEFD4FF47B
:10D8C00080742146044800F0ABF921460248BDE8C7
:10D8D0001040203000F0A4B9F8320020FF2803D80F
:10D8E0000146024800F0CBB900207047F832002012
:10D8F000FF2803D80146024800F0C1B90020704754
:10D900001833002010B50C46FCF790F8FF2804D01F
:10D91000024900EB400021F8204010BD28310020D2
:10D920001CB500F057F908B1F9F73EFA0020009055
:10D9300001909DF8000020F0720040F001003030AE
:10D9400020F080008DF8000007208DF801001020E5
:10D950008DF802009DF8030040F003008DF80300ED
:10D960009DF8040040F003008DF80400684600F0C4
:10D97000EBFA08B1F9F718FA064800F0CFFA08B147
:10D98000F9F712FA0448FBF765FD002801D0F9F712
:10D990000BFA1CBDDDDA0200499102000068012883
:10D9A00003D0022801D000207047012070470000FA
:10D9B0000449084490F93000082801DB0120704731
:10D9C00000207047983300200449084490F9300043
:10D9D000082801D2012070470020704798330020AA
:10D9E0002DE9F0410F46060026D0306820B370685C
:10D9F00010B3FF2400251CE02946706800F017F9D9
:10DA000048B1FF2C00D12C46281B401CB8420ED137
:10DA10002046BDE8F081FF2C06D108E021463046C3
:10DA200000F040F8641CE4B2AC42F7D3FF246D1C54
:10DA3000EDB2B068A842DFD8FF20EAE72DE9F04157
:10DA40000400DDE90705069E16D0A9B1A3B100FBCD
:10DA500005F7974210D8C21DB6EBD20F0CD358B1C0
:10DA600055B1E5602160C4E9013081B2184600F08B
:10DA7000D7F80020BDE8F0810720FBE770B504006F
:10DA80000D460DD0206858B1606848B1FF2D07D011
:10DA900000F0F5F820B1E168206805FB010070BDD9
:10DAA000002070BD70B504000D4611D0206800281C
:10DAB0000ED0606800280BD0FF2D09D000F0DFF8F1
:10DAC000002805D029466068BDE8704000F0E3B842
:10DAD00070BD002901D001F083B97047F8B5044644
:10DAE00000781E4D03260E281DD2DFE800F0071C2B
:10DAF0000F1C1D1C24351C331C352E35288818A1FD
:10DB000006EB0040BDE8F840FEF7A4B96088FAF7DC
:10DB10000DF80246207A00902888638806EB0040C2
:10DB20001AA1FEF7AAF9F8BD0020009060886946A6
:10DB3000FFF7CFFFF8BDFBF791FB0828FAD00028CC
:10DB4000F8D0BDE8F840F9F72FB9BDE8F84000205B
:10DB5000F9F748B82069F2E7A068F0E7F82D00204F
:10DB6000436F6E6E656374656420746F206120700E
:10DB7000726576696F75736C7920626F6E64656427
:10DB8000206465766963652E00000000436F6E6E49
:10DB9000656374696F6E20736563757265643A209E
:10DBA000726F6C653A2025642C20636F6E6E5F681F
:10DBB000616E646C653A20307825782C2070726F25
:10DBC0006365647572653A2025642E00FBF792BA8E
:10DBD000FBF790BA10B5FFF78FFC88B9FFF72EFB63
:10DBE00070B901F0FFF858B901F01AFA40B9FBF723
:10DBF000B9FE28B9FBF79EFF10B9FCF71BFA08B174
:10DC0000032010BD05484FF6FF718180002181601F
:10DC1000417001210170002010BD0000042C002083
:10DC2000002803D0C91DC908F8F747BC7047002871
:10DC300009D001F0070301229A40D2B200EBD100D3
:10DC40001146FCF7CFBD70472DE9F0410D460600A7
:10DC500013D0002401270EE004F0070007FA00F0BB
:10DC6000C1B206EBD400FCF7BDFD10B12046BDE803
:10DC7000F081641CA4B2AC42EED32846F7E740B171
:10DC800000EBD10001F0070200780121914008402B
:10DC900000D001207047F8B50400C1F3C70501F0BA
:10DCA00007014FF0010000FA01F0C6B20FD0605D2D
:10DCB00030420CD000208DF800006846F9F710F9CA
:10DCC000605DB04360559DF80000F9F72DF9F8BD8F
:10DCD0002DE9F041044686B001278088FCF778F9E9
:10DCE0006080207800263F4D082808D0092820D0E1
:10DCF0004FF6FF780A2829D00B2853D158E0607AD4
:10DD000010B1012809D04DE0A86830B1E168814226
:10DD100003D1AE60A088A88016E06878E8B3A08838
:10DD2000A98888423ED1207A06283BD100F08CFA9F
:10DD300038E0607A88BBA86878B3E168814231D165
:10DD4000AE60E868401EE860E6602BE0A878E8B1C5
:10DD50004046FFF79BFA4146404517D10846FFF77A
:10DD600093FA404512D1AE7014216846F8F7A5FB2E
:10DD70000C208DF80000ADF80480ADF8028000277B
:10DD80002046FBF7B7F96846FBF7B4F9687838B175
:10DD9000A088A988884203D100E003E000F054FA8B
:10DDA000002F1CD006B02046BDE8F041FBF7A2B919
:10DDB000A8780028F6D0AE7014216846F8F77DFBED
:10DDC0000D208DF80000ADF80480ADF80280A06849
:10DDD00002902046FBF78EF96846FBF78BF906B0F8
:10DDE000BDE8F081042C00200349097809B1FCF753
:10DDF0009DB9082070470000042C00202DE9FF4F3A
:10DE00002A4883B09946007892468B46B8B14FF6BF
:10DE1000FF763046FFF73AFA80460020009024480B
:10DE200001AA062100680190CDF808D04046FFF70E
:10DE30006BFA00256C1E3746072804D017E008202F
:10DE400007B0BDE8F08F0520FAE700200090A84257
:10DE500001D305464746A04201D204464646404605
:10DE6000FFF714FA804601AA0621FFF74DFAD8B150
:10DE70000528EAD0A8F57F41FF3901D00320DFE76C
:10DE80000399002001B10F80BBF1000F01D0CBF846
:10DE90000050BAF1000F01D0AAF80060B9F1000FEC
:10DEA000CED0C9F80040CBE70098D0E7042C002082
:10DEB0006800030070B5184E86B03078D0B10120EC
:10DEC000B0704FF6FF742046FFF7E0F90546A04218
:10DED0001DD10020B07014216846F8F7EEFA0C202E
:10DEE0008DF80000ADF80440ADF802406846FBF73D
:10DEF00001F90EE0082006B070BD00BFFFF774FF07
:10DF000008B10320F7E72846FFF7C0F90546A54208
:10DF1000F4D10020EFE70000042C0020084A11781B
:10DF200021B1D178032903D304207047082070471A
:10DF3000044B43F82100491CD170002070470000B9
:10DF4000042C0020383300200349097809B100F07F
:10DF50009BBF082070470000042C0020002801D03F
:10DF6000FBF7C8B8704770B50D00044602D1002019
:10DF7000F8F71AFF14B90020F8F716FF2878207078
:10DF800069886170090AA170A988E170090A217184
:10DF9000E8886071000AA07170BD000010B50C46E1
:10DFA000017A052908D0407A38B1084808A10268EA
:10DFB0002046FDF745F900E01AB106A12046FDF71D
:10DFC0003FF92046BDE81040FDF747B9842D0020F9
:10DFD000257300000D0A000038B5C3880D460446BD
:10DFE00033B114A0009015A216A12846FDF728F918
:10DFF000217A05291CD0607A48B1A088FDF7F4FD8C
:10E00000164951F8202016A12846FDF719F9A088D5
:10E010000021FDF7C7FF03461049207A143951F853
:10E02000202001B02846BDE830400EA1FDF708B918
:10E0300038BD00001B5B306D000000001B5B313BF6
:10E0400033316D0025734C6F67732064726F70708D
:10E050006564202825642925730D0A00842D00207D
:10E06000257300003C25733E2025733A20000000F4
:10E070000349884201D103487047002070470000DF
:10E0800000200040902C00200146054810B5006893
:10E09000FCF717FE04461C21F8F70FFA204610BDC6
:10E0A000F8000300014602480068FCF72BBE0000A0
:10E0B000F8000300034802490068FCF70DBE0000A9
:10E0C000282D002080010300F0B5254D254E85B098
:10E0D00004460027686828B9214930680831FCF7F0
:10E0E00006FE686001460078072817D2DFE800F0D6
:10E0F000160408080E0E12002046FCF773F802E022
:10E10000204601F083FE040028D008E02046FAF7FC
:10E1100053FEF8E72046FBF7CFFAF4E70F2414216B
:10E120006846F8F7CAF9A4F5E8501D3800D1002474
:10E13000019469466868FAF721FF6846FAF758FFC4
:10E1400007496F60002408313068FCF7C5FD0448BA
:10E1500001210C30FCF765FE0028BBD105B0F0BDF5
:10E16000E02C0020F80003002DE9F041234C0025AD
:10E17000234E207A012730B92248311D0068FCF770
:10E18000B6FD306038B1022020723168087928B1BC
:10E1900001281ED116E06560BDE8F081D1E90503D4
:10E1A000C01A4FF48052904200D31046B7EB900F44
:10E1B00001D2820800E001220869C96818441944A4
:10E1C00029DF03E0D1E90301084428DF58B1112811
:10E1D00012D003213068FAF71BFF25726560BDE895
:10E1E000F041FFF767BF207C0028D5D1BDE8F041A2
:10E1F00000210220FDF748BA2772CDE7E83600205B
:10E20000242D00208001030010B501210448FCF7F3
:10E21000EEFD002803D1BDE81040FFF755BF10BD4B
:10E22000EC2C002010B5074C201DFCF7D1FD002878
:10E2300006D1607C002803D1BDE81040FFF794BFF1
:10E2400010BD0000E8360020084910B500231A462A
:10E25000A1F10800FFF7D2FD30B1052804D000205D
:10E2600002490C39487010BD0120F9E7102C00203C
:10E2700010B510461A46F8F7F9F8002010BD000056
:10E280002DE9F0471B4F82460026387886B00028DB
:10E2900021D00024DFF86080A14600BF08EB041500
:10E2A000A87B810702D410EA0A0F1BD0012628465A
:10E2B00001F0A2FCB0B14FF6FF71ADF80210298851
:10E2C000ADF80410862809D007218DF800100290BF
:10E2D0006846FEF7A5FF06B0BDE8F08706208DF87A
:10E2E0000000F5E7641C022CD8D3002EF3D187F888
:10E2F0000090F0E7002C0020D83200202DE9F047F4
:10E3000007461E481C46154600780E4670B185B17A
:10E310007CB1DFF86C804FF00009A08802282BD276
:10E3200000EB800118F8210010BB19E00220BDE8C5
:10E33000F0870520FBE720681FB181883A88914269
:10E340000ED11EB101883288914209D180682860BF
:10E35000206868600A482830008928810020E6E7A4
:10E36000A088214600F05EF80028E4D1C4F80090AF
:10E37000A088401CA080D0E70A20D8E7002D00200C
:10E3800024360020F8B505464068244F0C46002688
:10E3900048B32349CA68824225D80969814222D3F9
:10E3A000FCF77CF8F8B12889398988421BD1D5E976
:10E3B00000018A68904216D10020A7F1280200BF10
:10E3C00000EB800302EB83035B688B4205D203F50D
:10E3D00080538B4201D9208011E0401C80B202287A
:10E3E000EED30020F8BD268000960AE00098296848
:10E3F0008068884205D100986860388928810120AA
:10E40000F8BD2088694600F00DF80028EED120887C
:10E41000401C80B220800228E6D3E2E74C36002080
:10E42000B02D002070B50E4600EB8001134800EBC4
:10E4300081004468306804F5805518B1418800EBCC
:10E44000810411E0083410E029462046FBF72AFC3D
:10E4500020B1012805D0022807D10DE00120346049
:10E4600070BD608804EB80040C3429462046FBF71D
:10E470002CFC0028E8D170BD002070BD243600209F
:10E4800038B50C460021009101460423074A08488C
:10E49000FDF74CF908B10E2038BD064A04EB8401A3
:10E4A00002EB810101200874002038BDFC0003004C
:10E4B000B02D0020243600200A46FF2803D801464C
:10E4C0001046FFF7E8BB7047084670471E4810B576
:10E4D0000078002837D01C481C49183000F0CBFACF
:10E4E00081B21B48F9F797FE17481849183000F019
:10E4F000C2FA81B21648F9F78EFE13481349183054
:10E5000000F0B9FA81B21248F9F785FE0E480F49BA
:10E51000183000F0B0FA81B20D48F9F77CFE0A48D5
:10E520000A49183000F0A7FA81B20948F9F773FEDA
:10E5300005480649183000F09EFA81B2BDE8104047
:10E540000348F9F768BE10BD902B0020E42F00208F
:10E55000882E002070B5012670044FF0E0210025C0
:10E56000C1F88001084C4010C4F84803C4F80803FF
:10E5700066602F20FEF706F9A660044C2F20A560E8
:10E58000FEF700F9A57070BD00100140B82C002006
:10E5900070B5054688690C4600284FF484712846FA
:10E5A0000AD0FEF7A4F8D5F81805626AE168885425
:10E5B000606A401C606270BDFEF799F8D5F81805D6
:10E5C00070BD1FB501238DF80030CDE90121D0E9E0
:10E5D0000012684690471FBD1FB501238DF800301B
:10E5E0008DF808100192D0E90012684690471FBDCF
:10E5F00010B50446064841792046F9F7C7FA0028C5
:10E6000004D12046BDE8104000F08EBA10BD0000D5
:10E61000DC2B002070B50D460446F8F785FA70B182
:10E620002846F8F793FA68B16807000E002C0CDA58
:10E6300004F00F0101F1E02181F8140D09E042F22C
:10E64000010070BD42F2020070BD04F1E02484F8C4
:10E650000004002070BD000038B50021012548B13C
:10E6600001280CD0032809D1FEF758F8BDE838403E
:10E67000FCF79ABD4FF0E020C0F8805138BD8DF80E
:10E6800000106846F8F72CFC064C207808B9FCF717
:10E690006FFDE068401CE060A5709DF80000F8F791
:10E6A00043FC38BD843300203EB504460949684622
:10E6B000FDF7CAFF08E000BFD0E9002120469047DF
:10E6C00030B16846FDF7D7FF02980028F4D13EBD6F
:10E6D00011203EBD500303003EB50446084968467C
:10E6E000FDF7B2FF07E000BFD0E9002120469047C8
:10E6F0006846FDF7C0FF02980028F5D13EBD000036
:10E700005C0303002DE9FC4104460C3000278046E1
:10E71000FBF730FD4FF6FF750646A842208803D16F
:10E72000FBF718FD064602E03146FBF7FDFC2088AA
:10E730000022012100F0C6F8AE4212D06A4607213D
:10E740003046FEF7E9FD60B9019D95F84400343587
:10E75000C00705D1414605F11200FBF7D0FC00B11E
:10E760002F46002320881A46394686DF05000BD045
:10E77000002320881A46314600F088F82088294670
:10E7800000F002F9BDE8FC81002FFBD100232088B6
:10E790001A46314600F07AF82088002241F206013C
:10E7A000FAF7C0FBEEE700002DE9FC411D46089C8E
:10E7B00016460F46804644B16B4601220721384673
:10E7C000FEF7D4FD112801D010B10320BDE8FC8173
:10E7D00050210198F7F771FE019806700198E560E5
:10E7E000343020600198183020610198401C60612D
:10E7F0000748E061019940461131FBF76DFB0028A5
:10E80000E3D107213846FEF73BFE0528DDD0DDE7E2
:10E8100044330020002835D00278910701D4110636
:10E820002FD4C2F3021104292BD8930703D503294F
:10E8300001D1110625D5437881788B4221D8072B49
:10E840001FD310291DD8C1784B071AD4007943076C
:10E8500017D40B0715D4030713D4D2074FEAC1729C
:10E8600001D042B10FE062B989070AD4C10708D1CB
:10E87000800706D407E0890705D4C10703D18007C4
:10E8800001D40020704701207047000070B50C468D
:10E8900005466AB1002B12D009480122C1782846EA
:10E8A000F9F78CF921462846BDE87040FBF73CBCDF
:10E8B000002B04D0BDE870400846FBF737BC70BDA4
:10E8C000142C0020F0B5174D14460F460A4685B0AB
:10E8D00006462978F9F772F9002F1FD00CB10122F2
:10E8E00000E0002269783046F9F768F9012C17D06A
:10E8F0000022A9783046F9F761F90022E97830461C
:10E90000F9F75CF9142208496846F7F7AFFDADF84E
:10E9100002608DF808406846FAF702FC05B0F0BDC9
:10E920000122E6E7142C00207C00030010B586B01D
:10E93000044614216846F7F7C0FD04208DF8000056
:10E94000ADF802406846FAF7EBFB06B010BD0000D8
:10E9500002498969002900D0084770479430002097
:10E9600030B585B00C460546142206496846F7F7CF
:10E970007DFDADF8025068460294FAF7ADFB05B094
:10E9800030BD0000B8FF020030B585B00C4605462A
:10E99000142206496846F7F769FDADF8025068464B
:10E9A0000294FAF7BDFB05B030BD000090000300F3
:10E9B0000348417881F0010141700248F9F746BCF3
:10E9C000902B0020882E002070B51548012451217D
:10E9D00064258460C0E9001504730146114800F005
:10E9E0003FF80F488C211030002601604FF49671DB
:10E9F00041600A218160067301460A48083000F030
:10EA00002FF807484FF4FA7120300560C0E901146F
:10EA100006730146BDE870400248103000F020B88F
:10EA2000C42F0020982B002010B503680A6889685D
:10EA30009C1A8C4202D9591A016010BD0121026052
:10EA4000017110BD10B54B68026889689C1A8C4230
:10EA500002D91144016010BD00210360017110BD95
:10EA60000A7B1AB149680160002102E0096801606F
:10EA700001210171704710B5044600790028204635
:10EA800002D0FFF7DFFF01E0FFF7CEFF206810BDE7
:10EA900070B50D4C0020D2B22070201D0B4D0378B4
:10EAA000EB5C1BB1001DFEF715F902E00C30FEF720
:10EAB00017F808B1F8F778F96078002802D02178C3
:10EAC0000029FAD070BD0000342D00207C2C0020DD
:10EAD0000348002201490079F9F712B8F1E5020074
:10EAE000DC2B00207CB50E490E4C0022D1E9000140
:10EAF000CDE900016946A088FEF733FC4FF6FF75AB
:10EB000007E00846FEF7C2FBA08000226946FEF738
:10EB100028FCA188A94201D01128F2D17CBD0000B7
:10EB20000C000300E82B002070B586B006460125D6
:10EB30000024FBF79BF8112812D005DCF0B1062861
:10EB400028D0082808D125E0A0F54051023907D087
:10EB5000A1F54071FF3924D001463046FFF700FF90
:10EB60002A46124D30462979F9F728F8697906B016
:10EB700022463046BDE87040F9F720B814220C490F
:10EB80006846F7F773FCADF8026001246846FAF7AF
:10EB9000A3FAE5E700253046FBF7DCFAFAF7BCFFFD
:10EBA000DEE73046FBF7E2FDDAE70000DC2B002071
:10EBB000E0FF02002DE9F0410746806A14468846CE
:10EBC000C8B3002531E000BFB96A05EB450001EB91
:10EBD0008006B088801CFE2802D90C20BDE8F08198
:10EBE0002288401C08F8020020881622401C80B2AF
:10EBF000208008F800202088401C80B2208000EB94
:10EC00000801308800F04EFE2188084480B2208040
:10EC1000B28842B1B16871B14044F7F727FC20884F
:10EC2000B188084420806D1CEDB297F82C00A842F2
:10EC3000CAD80020D2E7FFE70720CFE730B59DB064
:10EC40004E481A9000241AA94D48FCF714FA08B14E
:10EC5000F8F7AAF803208DF86C0014216846F7F73E
:10EC60002CFC1BA802909DF80C00012520F00F0041
:10EC7000401C20F0F00010308DF80C009DF80D00C5
:10EC8000009420F0FF008DF80D009DF80E008DF827
:10EC9000045020F0FF008DF80E009DF80F0069462B
:10ECA00020F00F00401C20F0F00010308DF80F0015
:10ECB0009DF8100020F0FF008DF8100030487838E3
:10ECC000F9F744FA08B1F8F76FF8142105A8F7F737
:10ECD000F4FB9DF82100059420F00F00401C20F06B
:10ECE000F00010308DF821009DF822008DF81850AA
:10ECF00020F00F00401C20F0F00010308DF82200B2
:10ED00009DF82300079420F0FF008DF823009DF864
:10ED1000240005A920F00F00401C20F0F000103066
:10ED20008DF8240064208DF8200015482838F8F765
:10ED300055FE08B1F8F738F840210AA8F7F7BDFBEF
:10ED400010A10AA8F9F785FA9DF8640020F00F00D9
:10ED5000401C20F0F00010308DF864009DF8650034
:10ED600020F0FF008DF865000AA8F8F781FF002861
:10ED700001D0F8F719F81DB030BD0000E1C1020064
:10ED8000002F00204E6F7264696353656D69636F75
:10ED90006E647563746F720010B50020F9F708FC9B
:10EDA00008B1F8F701F8F9F75DFB08B1F7F7FCFFD8
:10EDB00033DF002803D0BDE81040F7F7F5BF10BDE2
:10EDC00010B500F0ABF80548002203494078BDE8D3
:10EDD0001040F8F795BE000049A602001C2C002048
:10EDE00000F016B910B51148FAF799FB0F48401C0E
:10EDF000FAF795FB0D48801CFAF791FB0B48C01CF5
:10EE0000FAF78DFB0948001DFAF789FB0748401DFA
:10EE1000FAF785FB0548401E8179182903D00121A6
:10EE2000C171002010BD032010BD00001D2C00206A
:10EE300010B50078114C0A2813D004DC082810D033
:10EE400009281AD10DE00B280BD0132815D1002268
:10EE50000B49A079F8F754FE00220A49A078F8F788
:10EE60004FFE002206496079F8F74AFE6078BDE857
:10EE7000104000220349F8F743BE10BD1C2C0020AF
:10EE8000F1D1020049A6020070B50B4C05004FF00D
:10EE900001060CD0FFF7BEFC58B128682061287924
:10EEA000207504F11000A0602670002070BD0020C5
:10EEB000F9E7072070BD00001C2C002010B50446A7
:10EEC0000078052802D0122821D105E06088A168C9
:10EED000BDE8104000F060B90F480021806880B1A3
:10EEE0000D48237A1030007800F0010203B10123AD
:10EEF0009A4206D3627AC0F3400002B101229042E6
:10EF000000D20121608801230022FBF7FBFA204692
:10EF1000BDE81040FAF712B91C2C002030B50446A9
:10EF2000008885B014284FD00ADC11282CD0132873
:10EF300028D134F8040FF8F7F9FD01282FD038E074
:10EF4000192847D01A281DD1A088FEF74BF90028B0
:10EF500018D1A088F8F7C4FD0028A0884BD02A4912
:10EF600000220978F8F72AFE02208DF80000A08818
:10EF7000ADF8020000208DF808008DF80900684601
:10EF8000FAF7CEF805B030BD207A3D2804D04FF412
:10EF90008851A088002224E041F23D01F9E7207960
:10EFA000C00701D0012200E0022220880121FFF7E2
:10EFB00089FC34F8045B142214496846F7F756FAC2
:10EFC000ADF802500294DAE705B0201DBDE83040EC
:10EFD000FFF798BB217A201D41B14279008802F0E9
:10EFE000030205B0BDE83040FBF7E8BA05B0BDE864
:10EFF0003040F8F769B805B00122BDE8304041F271
:10F000000601F9F78FBF0000142C0020B8000300A0
:10F010000A7802490979F8F7D1BD0000142C0020C4
:10F0200010B51448FAF772FA1248401CFAF76EFA53
:10F030001048801CFAF76AFA0E48C01CFAF766FA04
:10F040000C48001DFAF762FA0A48017818290FD017
:10F05000417818290CD08178182909D0C17818294D
:10F0600006D00179182903D001214171002010BD7B
:10F07000032010BD142C002070B50C460546F8F78F
:10F0800055FD012802D043F2020070BD21004FF06F
:10F090000000FAD028467EDF70BD00002DE9F74F52
:10F0A0008AB0924688460A98F8F740FD06464FF621
:10F0B000FF7900244D4627460A98FEF73BFB83461E
:10F0C000202101A8F7F7F9F9012E01D0DEB105E002
:10F0D0002F48002201790A98F8F770FDB8F1000F67
:10F0E00016D098F80000C00714D00A98FBF732F841
:10F0F0000546484516D1FEF705F9054648450ED0A8
:10F100004FF0010B0CE043F202000DB0BDE8F08FB0
:10F11000852721E01F48CDF810A008901CE00324AB
:10F120006CB121E0012E0AD10A98F7F7ABFD30B996
:10F130000A98FFF7FBFB0A98F7F7A4FD50B101A866
:10F1400000905346324629460A98FFF72DFB0400EB
:10F1500002D009E0852712E0012E10D001AB002279
:10F1600039460A987FDF044654EA07000DD0002292
:10F170005B4629460A98FFF789FB2046C5E701ABA5
:10F18000424639460A987FDFEDE70122F0E70000AA
:10F19000142C0020443300203EB505460C4668463A
:10F1A000FBF752FD6A4621462846FEF724F8094837
:10F1B0000099C2682846FFF771FF04460146012204
:10F1C0002846FAF7C9F921462846009AF9F74AFF76
:10F1D0003EBD00001C2C0020002805D10349012061
:10F1E00048700020F9F726BC7047000084330020E7
:10F1F00010B51620F7F798FC48B10A4882684FF41A
:10F20000800152B1016821F48001016010BDBDE8A8
:10F21000104042F20100F7F7C7BD4FF0E020C0F800
:10F22000801110BD7035002010B51620F7F77CFC5A
:10F2300080B10F4890F800044009F7F787FC60B1EF
:10F240000C4882684FF480016AB1016841F4800182
:10F25000016010BD42F2010001E042F20200BDE88F
:10F260001040F7F7A1BD4FF0E020C0F8001110BD2D
:10F2700016E000E0703500202DE9F84F204D924651
:10F28000894606469846012269461846AF68F9F74E
:10F29000C5FA58B3009800210446801C09E000BF5D
:10F2A00000EA07035AF8212005EB8303401C491CA0
:10F2B000DA604145F4D34FEA164AF9F709FE4AEA03
:10F2C0000041601C384005EB80003C4005EB8402A7
:10F2D000C160D06866F3C50068F3891069F39F20A8
:10F2E00020F00300401C20F00400D06095F82004BA
:10F2F00002E000BFFCF79EFC0028FBD1BDE8F88FC0
:10F300000838002070B50C00054602D10020F7F740
:10F310004BFD15B90020F7F747FD207828702088AD
:10F32000000A68702068000CA8702068000EE87061
:10F3300020792871207A68712089000AA871A06854
:10F34000000CE87170BD00002DE9F84F1D4C002540
:10F350006846D4E901A6F9F7C5FD002738B30023B4
:10F36000009A61681CE0D1F800C00846944503D9B2
:10F37000ACEB02020A6015E0A2EB0C0263440760EA
:10F38000D0F80CC0C1698146BCF1000F08D006EB73
:10F39000030828F07F48C0E9018CC9F81C500546D5
:10F3A0000029E0D128466160FBF764F903E02846B4
:10F3B000FBF760F910B15046F9F75EFBE770BDE866
:10F3C000F88F0000B82C00200D4B10B5596831B1F2
:10F3D00002680C68A24204D8A21A0A60C16158608F
:10F3E00010BD0B4603E00B46C969121B21B10C6826
:10F3F0009442F8D3A41A0C600260C161D86110BDB8
:10F40000B82C00202DE9F041144E77683D462C467B
:10F4100003E0844204D02546E469002CF9D11BE0C6
:10F42000D4B1A5420BD1F869706040B90C490120F4
:10F4300088600021B160F0702F20FDF7A3F92168EA
:10F44000E069E86110B102681144016070688742A8
:10F4500002D00120BDE8F0810020FBE7B82C00209D
:10F46000001001407CB5064600240D468DF8004092
:10F470006846F7F735FD01A800F0E6FA70B10570AF
:10F48000094946609DF8040048709DF80000F7F7B0
:10F490004BFD1420F7F746F920467CBD04249DF867
:10F4A0000000F7F741FDF7E7643400202DE9F04153
:10F4B000194D6C68002C2CD0184800270068A968EA
:10F4C000B846401A20F07F462068B0420CD821464A
:10F4D000361A0744E469087C20B181F810808869F5
:10F4E00049698847002CEFD129786878814206D194
:10F4F000401CC0B26870022801D185F8018006481E
:10F5000069780C3040F82170BDE8F0411420F7F71D
:10F5100009B9BDE8F0810000B82C002004150140B5
:10F5200010B5F7F75FFC08B1F7F73EFC134A01216D
:10F530001348F7F745FC08B1F7F736FC1048114AB5
:10F540000121001DF7F73CFC08B1F7F72DFC0C4832
:10F550000D4A01210830F7F733FC08B1F7F724FC16
:10F5600007480A4A01210C30F7F72AFC002803D08B
:10F57000BDE81040F7F718BC10BD0000E9720200AA
:10F5800074FF0200DD9C0200CDE40200B1E902003C
:10F5900070B50C4605464FF48E71FDF7A8F8216A48
:10F5A000A068415C206A401C2062C5F81C1570BD33
:10F5B0001FB500228DF800200291816801914261FF
:10F5C000D0E90012684690471FBD00001FB50A46EB
:10F5D00001788DF8001041680191017A8DF80810CA
:10F5E000C0680390044850F82210001F50F82220F1
:10F5F000684690471FBD0000842C0020014901206F
:10F6000008707047342D002010B588B004462022C1
:10F610000E496846F6F72AFF06200090C01F0190A9
:10F62000029003904FF0EB7006900CB1084A00E096
:10F63000002269460748FBF7CFFD08B1F7F7B4FB96
:10F640000448001F447008B010BD00001C030300F4
:10F65000FDF50200382D00202DE9FF470C46054638
:10F660004FF40071FDF749F801274FF401780026A7
:10F6700018B34FF4927949462846FDF733F8E0B1C4
:10F6800049462846FDF733F8C5F8088394F8290061
:10F6900000B96F6002208DF80000D5F88004C5F82D
:10F6A00080040390A0690290E0680190A661E66181
:10F6B000D4E900126846904728E004212846FDF767
:10F6C0001CF818B34FF484712846FDF70BF8E8B125
:10F6D00021462846FEF75CFF616AA069884215D181
:10F6E000E06938B1E268616AA0612069E66166623A
:10F6F000E06008E094F8290000B96F60C5F808835D
:10F70000A661E268616A2046FEF75BFF4FF48E78DF
:10F7100041462846FCF7E6FF78B1206A61698842D5
:10F7200002D294F8280020B341462846FCF7DFFFB8
:10F73000616911B12046FFF73BFF4FF4A2784146C3
:10F740002846FCF7CFFF002818D041462846FCF792
:10F75000CEFF94F8290000B12F60A06900280DD0D9
:10F76000A661E268616A04B02046BDE8F047FEF792
:10F7700028BF21462846FFF70BFFDEE7BDE8FF87DD
:10F780001FB50A4601788DF8001041680191017A91
:10F790008DF80810C0680390044850F82210001F2C
:10F7A00050F82220684690471FBD0000842C00209E
:10F7B0002DE9FF410C464FF4927705463946FCF798
:10F7C000A2FF0026C0B139462846FCF7A1FF02205F
:10F7D0008DF80000D5F88004C5F880040390D5F8B2
:10F7E0003C058DF80800E0680190A661E661D4E967
:10F7F00000126846904723E04FF488773946284640
:10F80000FCF781FFE0B139462846FCF781FFD5F8C7
:10F810003C15A069884213D1E06960B1E268D5F86F
:10F82000000220F02000C5F80002E069A061206914
:10F83000E661E06001E0A661E2682046FEF7CCFEEA
:10F840004FF4A27739462846FCF75DFF60B1394690
:10F850002846FCF75DFFA06930B1A661D5F83C15DC
:10F860002046E268FEF7B8FE4FF490773946284606
:10F87000FCF749FF002813D039462846FCF748FF1B
:10F88000606900280CD0D5F84C058DF800608DF823
:10F890000800A06801906661D4E9001268469047AC
:10F8A000BDE8FF810870000A487002207047000020
:10F8B00010B514210448F6F700FE04480068FBF771
:10F8C000E5F9002010BD0000E836002080010300AB
:10F8D0002DE9F05F8346DDE90A4A994690460D46D8
:10F8E0000846012703E000BFB0FBF8F07F1C40454D
:10F8F000FAD2B94500D94F465FEACA7012D18CB12D
:10F900005FEA8A7002D5B9F1000F01D0202607E026
:10F91000302605E031465846641EF8F7C7FF0CB1A3
:10F92000A742F7D35FF00106B9F1010F02D9A9F19F
:10F93000010903E0B5FBF6F0404502D306FB08F6EB
:10F94000F2E7DFF83C9000BFB5FBF6F000FB165580
:10F9500019F800105846F8F7A9FFB6FBF8F6002E84
:10F96000F2D15FEACA7009D0002C07D0A74205D2B5
:10F9700020215846641EF8F799FFF5E7BDE8F09F8F
:10F98000100103000348002201498078F8F7B8B855
:10F99000398D0200DC2B0020F8B5054680B2FAF75D
:10F9A00085FC040013D0154E207A0027317B884255
:10F9B0000ED2A8B204F10A0175DF28B1112806D0D1
:10F9C000BDE8F840FEF7C4BF207A401C2072F8BDA5
:10F9D0002772307C38B1A8B23B2176DF18B10828F5
:10F9E00001D0FEF7B5FF71690029F0D08DF80070E5
:10F9F000ADF8025068468847F8BD000094300020FA
:10FA0000417939B190F8B21021B990F8B40008B139
:10FA1000012070470020704701460148FBF7BDB93F
:10FA2000B030002030B40446007A00280AD0608844
:10FA3000002166DF28B1112802D0616830BC084778
:10FA40000120207230BC70470A494A788B78521CDA
:10FA5000D2B2934200D100220B78934201D1002010
:10FA600070470270487800EB400001EBC000001DB9
:10FA700070470000643400202DE9FC411646DDE9A2
:10FA80000854CDE900541F468046022200F00CF8CD
:10FA9000002807D1CDE900543B46102231464046AC
:10FAA00000F002F8BDE8FC812DE9FC5F0026DDE9ED
:10FAB0000C4B994692468E4680462788354630E064
:10FAC000D8F80400002200EB850069460068019028
:10FAD00001A864DF002830D19DF8000050451FD1F7
:10FAE0000EB1002100E00221228808441118594576
:10FAF00022D846B9521C90B2208009F800E0208834
:10FB0000401C20800126218801A801EB09026946DA
:10FB100064DF002811D120889DF80010084420805F
:10FB20006D1CB8F80000A842CADC56B12088C01B82
:10FB3000401E80B2FF2802D90C20BDE8FC9F09F8C6
:10FB400007000020F9E710B5042817D209B10324F3
:10FB500000E00024F8F7D4FB4FF0A04101EB800057
:10FB6000D0F8001721F44031C0F80017D0F8001782
:10FB700041EA0441C0F80017002010BD062010BD66
:10FB8000002070472DE9F84F114D884681461E46EA
:10FB900017466946DDF828A02868FBF792F80400AC
:10FBA00013D01C21F6F789FC00202071C4F80090C6
:10FBB000C4E90486C4E902A769462868FBF7A2F8ED
:10FBC000FEF730FB0020BDE8F88F0420FBE70000C3
:10FBD0008001030082780121012A0BD0062A09D076
:10FBE000072A06D0082A06D1416889880931890880
:10FBF00000E01421018070471CB5044600200090ED
:10FC00000190A0788DF80200617B1A48FDF736FF5D
:10FC1000020017D0237BA1786846FDF791FD684666
:10FC2000FFF7D8FF208804F1080369466268FDF7F2
:10FC300005FD48B1072806D001210F4A112808D038
:10FC400086280FD003201CBDA17B21F00301A173E6
:10FC50001CBDA07B20F0010040F00200A0731170D9
:10FC600000201CBDA37B23F0020343F00103A37318
:10FC700011701CBDC8320020002C002038B505468C
:10FC80000C46002001E00098401C00906946284680
:10FC900000F00EF800280AD08178A142F3D1817BD0
:10FCA0008A07F0D4C907EED181680029EBD138BDAD
:10FCB00010B5084B0A6809E003EB0214248884425B
:10FCC00003D103EB02100A6010BD521C022AF3D3C9
:10FCD000002010BDD83200204FF6FF710180FF21B7
:10FCE00081704173817B21F00301817300210173D5
:10FCF000416081607047000070B50546002406E051
:10FD0000687B2044C1B20648FDF7CCFE641C287B0A
:10FD1000A042F5D82846BDE87040FFF7DDBF0000DF
:10FD2000C83200202DE9FC4706463648984614465E
:10FD300000780D464FF0000978B37DB32888A0F510
:10FD40007F41FF3931D0688848B36868FAF7A6FB6D
:10FD500068B374B32088ADF80000678801A8FEF787
:10FD600093F904002FD084F800804FF0000A84F843
:10FD700016A0BDF80000A08268682061214801211A
:10FD80000C38FBF728F8E060288820816888A0807C
:10FD9000E780B8F1030F1DD020E001E003E004E0AC
:10FDA0000220BDE8FC870520FBE70420F9E70320DB
:10FDB000F7E7FFE72889694687B2384600F0ACF8D4
:10FDC0000028EED1CAE7BDF80010384600F098F8D8
:10FDD0000820E6E70420A0753068A061A4F80A9026
:10FDE00001A8FEF75FF946B1C6F804A0E16806482D
:10FDF000316086F80AA000893081FEF705FA0020FC
:10FE0000CFE70000002D00204C3600202DE9F843FC
:10FE10000D46898A374A01EB810102EB810630B138
:10FE200029463046FDF7ECF80120BDE8F88331891A
:10FE30007068002400EB81072E48A97DA8384FF098
:10FE40000E0807294ED2DFE801F00D2D16240440DC
:10FE50004A004460A969016026482749A838FEF78E
:10FE600091FA30B10220A875042339462A1D009466
:10FE700023E00A20D9E728692A4608B1032000E0D8
:10FE800001209075042305F10C0207F1080100948C
:10FE900013E00120A8750094E88807F10C018300A5
:10FEA0002A690AE028782A4603280CD00620907593
:10FEB000042305F10802391D00941048FBF736FCB5
:10FEC000A8B144460FE00520F1E70621A9750A49CB
:10FED00040680988FEF7D4FA040004D107E041F62F
:10FEE0001D5400E00F2429463046FDF789F82046CE
:10FEF0009BE7000024360020E02C0020B02D0020DD
:10FF000001EB8102034901EB82014A89101AC01EEC
:10FF1000488170472436002070B5C01C82B240F280
:10FF2000FE30824201D3092070BD114B00204FF4F6
:10FF3000806500BF00EB800413F8246096B903EBE2
:10FF400084063489768914443444A4B2AC4209D27C
:10FF5000088000EB800003EB80004189114441815F
:10FF6000002070BD401C80B20228E3D3072070BD82
:10FF700024360020082E0020282E0020482E0020A5
:10FF8000682E0020111213140D0E0F10F42F0020F4
:10FF900014300020403000200D0003008584020052
:10FFA0000E000300858402000F0003008584020018
:10FFB000100003008584020007000000000000001C
:10FFC000000000000000000000000000060000002B
:10FFD0000000000000000000000000000000000021
:10FFE0001000000000000000000000000000000001
:10FFF00000000000110000000000000000000000F0
:020000040003F7
:1000000000000000000000000100000001000100ED
:1000100008000300010001001C00030000000000B4
:10002000D1DB020035990200770A000000000000D1
:10003000770A0000000000007ADA000000000000EB
:1000400091D2020007000000000000000000000044
:100050000000000000000000D1DC020031EE0200D0
:10006000359C0200B599020001000000000000006C
:1000700001000600102C0020BDEE0200010000006F
:100080000000000000000000000000000000000070
:100090000700000000000000000000000000000059
:1000A000000000000300000000000000000000004D
:1000B000000000000000000005000000000000003B
:1000C0000000000000000000000000005DDF0200F2
:1000D00000000050FDC9020059CC020003000000DE
:1000E0004434002000000000000000000000000078
:1000F0000338FDD870470000CC2C00200000FFFF23
:10010000DEC0ADDEFF011EF1DEC0ADDEFE011EF180
:10011000303132333435363738394142434445463D
:100120006E72665F6673746F726167655F696E6930
:1001300074006E72665F6673746F726167655F7577
:100140006E696E6974006E72665F6673746F726159
:1001500067655F72656164006E72665F6673746F77
:10016000726167655F7772697465006E72665F665B
:1001700073746F726167655F65726173650000001B
:10018000102D0020001000000400000001000000FD
:10019000B1A10200B1F8020071E2020085FB020089
:1001A000318F0200C9E4020081FB020035A4020085
:1001B000000000000000000000000000000000003F
:1001C0000000000000000000B0010300C8010300AF
:1001D00004000000556E6B6E6F776E206572726F53
:1001E0007220636F6465000000000000D408030003
:1001F00001000000800703000200000074050300F6
:1002000003000000F4070300040000004808030096
:10021000050000002807030006000000C4060300D4
:100220000700000030080300080000003C0703003E
:1002300009000000A00703000A000000BC0803003A
:100240000B0000005C0503000C00000054070300D5
:100250000D000000240903000E0000002008030028
:100260000F0000005C08030010000000900803006D
:100270001100000038090300120000000C090300FF
:1002800013000000A808030080000000DC06030043
:10029000810000001806030082000000D80503005A
:1002A00083000000B805030084000000F40503008B
:1002B0008500000000070300860000000808030016
:1002C00090000000A40603009100000098050300C0
:1002D000920000006807030000820000700803001D
:1002E00001820000BC07030002820000D80703005F
:1002F000008400003406030001840000E0080300CD
:10030000028400007C0603000384000058060300FA
:10031000D1BB0200A5BB02009DBB0200FFFFFFFF97
:10032000FFFFFFFFFFFFFFFFFFFFFFFF00000000D9
:10033000000000000000D60107010000480D030086
:10034000500D030000000000000000000100000745
:100350003C0303004C030300080000007403030087
:1003600084030300080000008403030094030300D7
:1003700008000000780D0300880D03000000000055
:1003800000000000680D0300780D0300000000006D
:1003900000000000F80C0300000D0300000D030036
:1003A000280D0300280D0300400D0300400D03003D
:1003B000480D0300902B002094030300B4030300B6
:1003C00008000000500D0300600D0300600D0300E5
:1003D000680D0300C4030300D403030008000000F9
:1003E0000040404040404040404041414141414048
:1003F00040404040404040404040404040404040FD
:10040000400502020202020202020202020202028B
:100410000220202020202020202020020202020290
:1004200002029090909090901010101010101010E8
:1004300010101010101010101010101002020202F4
:100440000202888888888888080808080808080838
:100450000808080808080808080808080202020234
:1004600040000000E103030073645F626C655F6736
:1004700061705F646174615F6C656E6774685F75FD
:1004800070646174652829202872657175657374BC
:1004900029206F6E20636F6E6E656374696F6E20C6
:1004A000307825782072657475726E6564202573C6
:1004B0002E0000005468652072657175657374655F
:1004C0006420636F6D62696E6174696F6E206F6620
:1004D00020545820616E64205258207061636B650F
:1004E00074206C656E6774687320697320746F6F15
:1004F000206C6F6E67206279202575206D696372AC
:100500006F7365636F6E64732E00000061646472C4
:100510005F69735F77697468696E5F626F756E6437
:100520007328705F66732C20706167655F61646417
:10053000722C20286C656E202A20705F66732D3E19
:10054000705F666C6173685F696E666F2D3E657281
:100550006173655F756E6974292900004E52465FAC
:100560004552524F525F494E56414C49445F4441B7
:10057000544100004E52465F4552524F525F534F16
:1005800046544445564943455F4E4F545F454E419E
:10059000424C4544000000004E52465F4552524FC7
:1005A000525F464541545552455F4E4F545F454E4C
:1005B00041424C45440000004E52465F4552524F66
:1005C000525F4D555445585F554E4C4F434B5F4617
:1005D00041494C45440000004E52465F4552524F3F
:1005E000525F4D555445585F4C4F434B5F46414910
:1005F0004C4544004E52465F4552524F525F4D5556
:100600005445585F434F4E445F494E49545F4641FD
:10061000494C4544000000004E52465F4552524F3F
:10062000525F4D555445585F494E49545F464149C4
:100630004C4544004E52465F4552524F525F424C29
:10064000455F495053505F52585F504B545F54526E
:10065000554E4341544544004E52465F4552524F19
:10066000525F424C455F495053505F504545525F81
:1006700052454A4543544544000000004E52465FEF
:100680004552524F525F424C455F495053505F4C68
:10069000494E4B5F444953434F4E4E4543544544A6
:1006A000000000004E52465F4552524F525F41508B
:1006B000495F4E4F545F494D504C454D454E544552
:1006C000440000004E52465F4552524F525F4E4F1B
:1006D000545F535550504F52544544004E52465F5C
:1006E0004552524F525F4D4F44554C455F4E4F540B
:1006F0005F494E495449414C495A45440000000065
:100700004E52465F4552524F525F4D4F44554C45F5
:100710005F414C52454144595F494E495449414C0F
:10072000495A4544000000004E52465F4552524F20
:10073000525F4E4F545F464F554E44004E52465FF7
:100740004552524F525F494E56414C49445F5354B3
:10075000415445004E52465F4552524F525F44410C
:1007600054415F53495A45004E52465F4552524FDD
:10077000525F494F5F50454E44494E4700000000CC
:100780004E52465F4552524F525F5356435F484167
:100790004E444C45525F4D495353494E470000006B
:1007A0004E52465F4552524F525F494E56414C4958
:1007B000445F4C454E475448000000004E52465F8F
:1007C0004552524F525F4452565F5457495F45520B
:1007D000525F414E41434B004E52465F4552524F8D
:1007E000525F4452565F5457495F4552525F444EE0
:1007F00041434B004E52465F4552524F525F494E65
:100800005445524E414C00004E52465F4552524FA5
:10081000525F53544F524147455F46554C4C000080
:100820004E52465F4552524F525F4E554C4C00005F
:100830004E52465F4552524F525F494E56414C49C7
:10084000445F504152414D004E52465F4552524F17
:10085000525F4E4F5F4D454D000000004E52465FC7
:100860004552524F525F464F5242494444454E0012
:100870004E52465F4552524F525F4452565F545754
:10088000495F4552525F4F56455252554E00000047
:100890004E52465F4552524F525F494E56414C4967
:1008A000445F4144445200004E52465F4552524F0D
:1008B000525F5245534F5552434553004E52465F87
:1008C0004552524F525F494E56414C49445F464C47
:1008D000414753004E52465F5355434345535300DF
:1008E0004E52465F4552524F525F424C455F49500F
:1008F00053505F4348414E4E454C5F414C52454139
:1009000044595F4558495354530000004E52465FC6
:100910004552524F525F434F4E4E5F434F554E54D8
:10092000000000004E52465F4552524F525F5449FC
:100930004D454F55540000004E52465F4552524FB0
:10094000525F4255535900007761726E696E6700BD
:1009500064656275670000001B5B313B33306D00DE
:100960001B5B306D000000001B5B313B33316D00C1
:100970001B5B313B33326D001B5B313B33336D000E
:100980001B5B313B33346D001B5B313B33356D00FA
:100990001B5B313B33366D001B5B313B33376D00E6
:1009A000696E666F000000006572726F7200000071
:1009B00073645F626C655F6366675F736574282943
:1009C0002072657475726E65642025732077686582
:1009D0006E20617474656D7074696E6720746F2029
:1009E00073657420424C455F47415454535F4346FE
:1009F000475F534552564943455F4348414E47453B
:100A0000442E000073645F626C655F6366675F73AA
:100A1000657428292072657475726E65642025736B
:100A2000207768656E20617474656D7074696E6797
:100A300020746F2073657420424C455F434F4D4DC9
:100A40004F4E5F4346475F56535F555549442E000E
:100A500073645F626C655F6366675F7365742829A2
:100A60002072657475726E656420257320776865E1
:100A70006E20617474656D7074696E6720746F2088
:100A800073657420424C455F47415454535F43465D
:100A9000475F415454525F5441425F53495A452E77
:100AA0000000000073645F626C655F6366675F737C
:100AB000657428292072657475726E6564202573CB
:100AC000207768656E20617474656D7074696E67F7
:100AD00020746F2073657420424C455F434F4E4E27
:100AE0005F4346475F4741502E00000073645F62DA
:100AF0006C655F6366675F7365742829207265742F
:100B000075726E6564202573207768656E20617448
:100B100074656D7074696E6720746F2073657420DE
:100B2000424C455F4741505F4346475F524F4C45FB
:100B30005F434F554E542E0073645F626C655F6374
:100B400066675F73657428292072657475726E65B7
:100B500064202573207768656E20617474656D70FC
:100B600074696E6720746F2073657420424C455F12
:100B7000434F4E4E5F4346475F474154542E00005B
:100B80006E72665F626C655F67617474000000007E
:100B9000626C655F62617300636C6F636B00000081
:100BA000434C4F434B0000004750494F5445000011
:100BB00050525300554152540000000055415254C8
:100BC0004500000061746669666F2E6D5F71756522
:100BD000756500006E72665F6673746F726167653B
:100BE0000000000061746669666F2E6D5F6669665D
:100BF0006F0000007077725F6D676D740000000019
:100C000062616C6C6F632E6C6F675F6D656D706F8A
:100C10006F6C0000617070006E72665F73646800D4
:100C20006E72665F7364685F626C65006E72665FA9
:100C30007364685F736F6300880D0300902B00205E
:100C4000780200003C650200F00D0300082E002031
:100C5000282E0000186B0200800B03000000030325
:100C6000900B030000000000980B03000000000040
:100C7000A00B030000000000A80B03000000000010
:100C8000B00B030000000000B40B030000000000E4
:100C9000BC0B030000000000C40B030000000003B5
:100CA000D40B030000000303E40B03000000000367
:100CB000F40B030000000000000C03000000000320
:100CC000140C030000000303180C030000000303CE
:100CD000200C0300000003032C0C0300000003039E
:100CE000602D0020582D0020602D00204837002066
:100CF000F42D002018000000C57F02000000000055
:100D000019AF0200EC2E0020117602000C2F0020FB
:100D1000597E020000000000C97E020000000000B1
:100D2000C980020000000000AB810200882E002074
:100D30001B7A0200D82E00209BB00200002F00205A
:100D40009D7D02000000000051B60200000000007E
:100D5000D9F102000000000089B602000000000086
:100D60007B7602000C2F00207DC4020000000000F2
:100D70000DC602000000000059E60200000000005D
:100D800069B60200000000001201031CFFFF140DF1
:100D900018011A0F041A0A040128042DCDDB022AB7
:100DA00018017909390A01B513E42D0240200A1A05
:100DB000EC441220AA4008042510030314A80903D8
:100DC0001A48041AA0041A50041A60041A58041A83
:100DD00068041A70041A78041A80041A88041A9095
:100DE000041A9804517B90D061044DDD95020000F7
:040000050002620192
:00000001FF
